:020000040800F2
:10000000B08B002081020008232D0008972B0008E8
:10001000212D00085B120008A52E0008000000003A
:10002000000000000000000000000000272D000874
:10003000EB13000800000000252D0008292D000802
:100040009B0200089B0200089B0200089B0200081C
:100050009B0200089B0200089B0200089B0200080C
:100060009B0200089B0200089B0200089B020008FC
:100070009B0200089B0200089B0200089B020008EC
:100080009B0200089B0200089B0200089B020008DC
:100090009B0200089B0200089B0200089B020008CC
:1000A0009B0200089B0200089B0200089B020008BC
:1000B0009B0200089B020008D12D00089B0200084B
:1000C0009B0200089B0200089B0200089B0200089C
:1000D0009B0200089B0200089B0200089B0200088C
:1000E0009B0200089B0200089B0200089B0200087C
:1000F0009B0200089B0200089B0200089B0200086C
:100100009B0200089B0200089B0200089B0200085B
:100110009B0200089B0200089B0200089B0200084B
:100120009B0200089B0200089B0200089B0200083B
:100130009B020008851400089B0200089B0200082F
:100140009B0200089B0200089B0200089B0200081B
:100150009B0200089B0200089B0200089B0200080B
:100160009B0200089B0200089B0200089B020008FB
:100170009B0200089B0200089B0200080000000090
:100180009B0200089B02000800F002F800F04EF805
:100190000AA090E8000C82448344AAF10107DA45E2
:1001A00001D100F043F8AFF2090EBAE80F0013F0E6
:1001B000010F18BFFB1A43F00103184774C1000078
:1001C00094C10000103A24BF78C878C1FAD8520709
:1001D00024BF30C830C144BF04680C6070470000C1
:1001E0000023002400250026103A28BF78C1FBD840
:1001F000520728BF30C148BF0B607047642900F028
:100200004181732900F0C182002070471FB50BF0B7
:1002100061FF9DE8030000F015FE00F084F900F096
:100220001DFB1FBD10B500F082FB10BD00F0E5FB0B
:100230001146FFF7EBFF05F004F800F0D5FD03B41D
:10024000FFF7F0FF03BC00F077FF00000B49D1F887
:1002500000C04A685CF8043B1068184442F8040B7C
:100260008C4528BFA1F1DC0C8A4228BFA1F1DC0239
:10027000C1F800C04A6020F0004070474884002068
:100280000948804709480047FEE7FEE7FEE7FEE72A
:10029000FEE7FEE7FEE7FEE7FEE7FEE70448054966
:1002A000054A064B70470000C12D0008890100086F
:1002B000B0850020B08B0020B0870020B0870020E0
:1002C00053EA020C00F069802DE9F04B4FF0000674
:1002D000002B1FBFB3FA83F503FA05F424FA05F6E1
:1002E0005E4012BF1643B2FA82F502FA05F4C5F178
:1002F00020051EBF22FA05FC44EA0C04203556EA0C
:10030000044C4FEA144418BF641C4FF000084FF02F
:100310000009904271EB030C39D3002919BFB1FADF
:1003200081F701FA07F6B0FA80F700FA07F6C7F18D
:1003300020071EBF20FA07FC46EA0C062037B6FB52
:10034000F4FCA7EB0507103F07F01F0BCBF12006CD
:100350000CFA0BFB2CFA06F644BFB3460026202FFE
:10036000A4BF5E464FF0000B5BEA060C08BF4FF0DF
:10037000010B19EB0B09ABFB027C48EB0608C01B19
:1003800006FB02CC0BFB03CC71EB0C01C1E70B4667
:10039000024641464846BDE8F08B13B54FF00000D9
:1003A0004FF00001AFF30080BDE81C407047000033
:1003B0000FB4044910B503AA029800F0EBF910BC81
:1003C0005DF814FBA48400202DE9F0410E4604469C
:1003D000002020622046E168884730B3252805D0F8
:1003E000D4E901219047206A401CF2E7E1682046E9
:1003F00000278847050018D0A5F14100192802D828
:1004000020354FF400673246294620462760FFF723
:10041000F5FE40B1012804D0F61D26F00706083687
:10042000D8E7361DD6E72846DAE7206ABDE8F0812E
:1004300070B50C460546012A05D02878800600D5FF
:10044000EA69002302E0012305E05B1C934202D22B
:10045000E05C0028F9D1A869E618C01AA861286AEA
:10046000184428622846AFF3008004E0D5E9012152
:1004700014F8010B9047B442F8D32846AFF300803C
:1004800070BD00002DE9F041064600241068752972
:10049000314616A510D0AFF30080002802DA4042A2
:1004A00013A507E031688A0701D512A502E04907C4
:1004B00004D511A5012401E0AFF3008000210A2238
:1004C00006F1240709E0B0FBF2FCB0FBF2F302FBFB
:1004D0001C00303078541846491C0028F3D12346BC
:1004E0002A463046BDE8F04100F0E4B800000000C4
:1004F0002D0000002B000000200000000B4910B56B
:10050000A1F17C020A4CC2E93712372106E000EB68
:10051000104342F82130074B00FB03400B1EA1F1B2
:100520000101F4DC10BD0120E8E70000E8830020B1
:10053000E119D666CD0D010040EA010310B59B0715
:100540000FD1042A0DD310C808C9121F9C42F8D03D
:1005500020BA19BA884201D9012010BD4FF0FF30EE
:1005600010BD1AB1D30703D0521C07E0002010BD04
:1005700010F8013B11F8014B1B1B07D110F8013B90
:1005800011F8014B1B1B01D1921EF1D1184610BD71
:1005900010B5431C02E010F8011B71B18107FAD1BC
:1005A0004FF0013202C88C1A8C4314EAC211F9D000
:1005B000C01A0A0603D0C01E10BDC01A10BD0A041E
:1005C00001D0801E10BD0902FCD0401E10BD032AC0
:1005D00040F2308010F0030C00F0158011F8013B60
:1005E000BCF1020F624498BF11F801CB00F8013B47
:1005F00038BF11F8013BA2F1040298BF00F801CB0B
:1006000038BF00F8013B11F0030300F0D580083A31
:10061000C0F0088051F8043B083A51F804CBA0E838
:100620000810F5E7121D5CBF51F8043B40F8043B8D
:10063000AFF30080D20724BF11F8013B11F801CBC2
:1006400048BF11F8012B24BF00F8013B00F801CB93
:1006500048BF00F8012B70474FF0000200B5134669
:1006600094469646203922BFA0E80C50A0E80C50D2
:10067000B1F12001BFF4F7AF090728BFA0E80C5083
:1006800048BF0CC05DF804EB890028BF40F8042B7C
:1006900008BF704748BF20F8022B11F0804F18BFE9
:1006A00000F8012B7047704770477047004870474B
:1006B0004C8500202DE9F0470D46994692460446A8
:1006C00000F124080168880604D5E06921F01001D2
:1006D000216000E00120A84201DD471B00E0002767
:1006E000A1697A1902EB0900081AA0612078C006F6
:1006F00002D42046AFF30080002608E0D4E90121AF
:100700001AF806009047206A401C761C20624E456D
:10071000F4DB2078C0060AD52046AFF3008006E05F
:10072000D4E9012130209047206A401C2062381E05
:10073000A7F10107F4DC07E0D4E9012118F805006E
:100740009047206A401C2062281EA5F10105F3DCB9
:100750002046AFF300802078000602D50220BDE8D5
:10076000F0870120FBE710B5436913B1AFF30080B8
:1007700001E0FFF75DFE012010BD127800F12401B9
:100780000A7000224A700122EDE711684FF0FF3233
:10079000E9E70000074B70B50D467B4400F047F8D1
:1007A0000446284600F056F810B14FF0FF3070BDF7
:1007B000204670BDA736000010B5203AC0F00B806F
:1007C000B1E81850203AA0E81850B1E81850A0E855
:1007D0001850BFF4F5AF5FEA027C24BFB1E81850AF
:1007E000A0E8185044BF18C918C0BDE810405FEA1F
:1007F000827C24BF51F8043B40F8043B08BF70479B
:10080000D20728BF31F8023B48BF11F8012B28BF9F
:1008100020F8023B48BF00F8012B704700487047A2
:100820004C85002001694A1C02610878704700B5B8
:100830008FB0CDE901310021059105497944CDE919
:10084000031011466846FFF7BFFD0FB000BD000062
:10085000E5FFFFFF007B00F08000704710B54248C5
:100860005421FFF7F9FE41485421FFF7F5FE4048B7
:100870005421FFF7F1FE3F493B483C4A3F4B08609B
:100880003D490A603A491960531C0365481C1065CC
:10089000012008653B48344A39A1784400F008FA41
:1008A00020B9384878440A3800F0A7FA37482F4A68
:1008B00035A1784400F0FCF920B9344878440A386E
:1008C00000F09BFA32482A4A2FA1784400F0F0F950
:1008D00020B92F4878440A3800F08FFA4023224884
:1008E000DC000021224600F0BFF920B12548784401
:1008F000543800F082FA1D4822464023002100F0BF
:10090000B3F920B121487844543800F076FA1848F9
:1009100022461023002100F0A7F9002806D01C4829
:100920007844BDE81040563800F067BA10BD104852
:1009300070B5006D20F001040B4800F02FFA0B4851
:1009400000F02CFA0A4800F029FA09E0206D20F0A6
:100950000105204600F022FA204600F073F82C46EC
:10096000002CF3D170BD000050840020A48400202E
:10097000F8840020EC000020F0000020F4000020AB
:100980007200000072B90000770000005EB900003C
:100990004AB900000EB5CDE90001FFF7F9FD02905C
:1009A00069460120ABBE0EBD08B569460090022025
:1009B000ABBE08BD1FB58DE8070069460520ABBE7C
:1009C00004B010BD1FB58DE80F0069460620ABBE10
:1009D000F6E708B5694600900920ABBE08BD1CB516
:1009E000CDE9000169460A20ABBE1CBD704708B5C1
:1009F000694600900C20ABBE08BD7546FFF70EFFA0
:100A0000AE4605006946534620F00700854618B0FB
:100A100020B5FFF743FCBDE820404FF000064FF043
:100A200000074FF000084FF0000B21F00701AC4623
:100A3000ACE8C009ACE8C009ACE8C009ACE8C00942
:100A40008D46704770B50446051F00F0DFF9006859
:100A5000002C14BF446870BD002C18BFAC423CBFD2
:100A600020466468F8D301680A18AA4218BF456096
:100A700003D12A6805461144016028684119A14242
:100A80001CBF6C6070BD61686960216808442860A3
:100A900070BD2DE9F04705460C46C86820F42010CB
:100AA00040F48000C860800602D5084600F0FBFADA
:100AB000E06841F282014FF0FF390140022903D082
:100AC000204600F099FAB5E000F42041B1F5004F5E
:100AD0000FD1C00306D56168E06A884200D8084695
:100AE000606006E02069E06260606069FFF77FFF98
:100AF000A061A0680022EEB200280DDAE1688B0543
:100B00000AD4C043A06041F490302260E060606885
:100B1000411C61600670A5E0E0689046226040F4E8
:100B20000050E060206968BB6069FFF752FF012751
:100B300004F12405A0B1A08910F4407F08D0E06939
:100B400000F0AFF9206118B1E06840F4006016E0F1
:100B5000E7612561E06820F4407040F480600EE0B9
:100B6000E06900F09EF900282061F1D0E06840F4CF
:100B7000006010F4407FE06002D140F48070E060DB
:100B800020696060E06825696FF0010AC1051FD522
:100B90006168E06A884200D80846411B04D02246BA
:100BA000284600F033FAF0BBE068010203D5E562A5
:100BB000C4E9015854E0691CE1626160E16940F4F4
:100BC0008030491EC4E9021030462E70BDE8F0871F
:100BD000010202D500F480320AE06068411C6160C5
:100BE0000670E0680A2E40F48030E06006D00022F3
:100BF000E16A6068814203D90B4602E00122F7E70F
:100C00000346A7895B1B7F0503D4E7699F4200DD8C
:100C1000E2B1814200D80146E5620F1AC4E90158E9
:100C2000002B09DD00E005E022461946284600F0C9
:100C3000EDF908B14846C9E747B1A069E5626560CA
:100C4000C01BA061E06840F01000E060E0680002B6
:100C500008D56168A069E562491B08446560A06128
:100C60005046B3E73046B1E770B5C468A50713D066
:100C7000650211D4B2F5807F09D0B2F5007F06D0AD
:100C8000B2F5806F08D1012300F1240106E05D1E5A
:100C90006FF07F46B54201D3012070BD0161C36191
:100CA000416024F470611143C160002070BD0000F8
:100CB0002DE9F0410C4607461646104600F06EF846
:100CC0002078611C61280AD0722802D077283CD194
:100CD00002E00125002405E00225042402E00824A6
:100CE00048F2020511F8010B2B2806D0622809D022
:100CF00011F8010C74280AD00BE045F0030544F00C
:100D00000204EFE745F0040544F00104EAE744F08B
:100D1000100438462146FFF73DFE411C15D0002146
:100D2000316171604FF40071F560F161706120070D
:100D300004D530460222002100F0E2F8306D40F088
:100D4000010030653046BDE8F0810020FBE72DE969
:100D5000F0410D460646104C206DC10704D04108F5
:100D600004D020F00104F7E722460EE0542000F002
:100D700098F807000ED0206D47F001010843542178
:100D800020653846FFF768FC3A4629463046BDE8FC
:100D9000F0418DE70020D6E7508400202DE9F04790
:100DA00004464FF000094FF0FF37C568D4E90486C8
:100DB000A80707D0204600F053F93046FFF7F4FDAE
:100DC000002802DA3846BDE8F087280502D54046FB
:100DD000FFF738FE4C212046FFF73EFC206D20F047
:100DE000010020654846EEE710B50446AFF30080E9
:100DF0002046BDE81040FFF722BA10B500F07AF99E
:100E0000BDE8104000F070B970470000004870471E
:100E100054850020704770477047704738B50446C6
:100E20000A4600206946AFF30080002808BF38BD9D
:100E300002460099204600F08CF9012038BD0120BF
:100E400000F072B9F8B5AFF30080054600200C46FB
:100E5000102000BF0646A819A0420DD932466946A7
:100E60000020AFF30080070008BF00F05DF9009894
:100E7000A04218BF0546C419FFF7C8FF0560074622
:100E8000F01D20F007004619284600F05BF9B44237
:100E900008BFF8BDA21B31463868BDE8F84000F035
:100EA00058B970B50646FFF7B1FF056806F10B00AB
:100EB00020F00704B4429CBF002070BD2B466A6836
:100EC000BAB11068A04210D304F1080188423CBFB7
:100ED0005068586007D35168101941601168091BA8
:100EE000016058601460101D70BD13465268002ADE
:100EF000E7D121462846FFF791FF0028DED170BDDB
:100F00002DE9F041044616460D464769007B8007EF
:100F10002ED03846FFF75DFD50BB3EB3012E02D008
:100F2000022E25D104E0204600F02DF905441DE0F5
:100F30003846FFF75CFDE168002841F01001E160F0
:100F400005DA204600F058F80120BDE8F081C90319
:100F50000BD56268E16A914200D81146A26911443A
:100F60002269891A814200DD08460544002D01DA14
:100F70000220EAE7E16A6068E268814206D29103F2
:100F8000E06203D522F4003141F01002A669002787
:100F9000AE4213DCE16A814201D90B4600E0034610
:100FA00003EB060C2369ACEB030CAC4506DD814278
:100FB00001D98C4600E084469C4505D1A760276096
:100FC00042F02000A5620DE0AD1BE669AE1B814238
:100FD000A66000D90846C01A281A20605819606017
:100FE00022F0200003490840E060002084F84870A7
:100FF000ABE70000BFCFD7FFC16821F4001141F07B
:101000008001C16000218160016070472DE9F047D7
:10101000814614460E464FF0FF383248D56857696E
:10102000054209D03846A169FFF7D9FC002811DB39
:101030002C48C0430540E5602B46324649463846B9
:10104000FFF7B8FCA16920F00042B21A1144002851
:10105000A16103D02046FFF7CFFF4046BDE8F087EF
:1010600070B504460569C06A6168884200D80846C0
:10107000E16821F42011E160C90312D5A84208D02B
:101080002246411B2846FFF7C1FF10B14FF0FF3049
:1010900070BD0020E562C4E90150E06820F48030B2
:1010A000E060002070BD10B50446C06820F020004C
:1010B000E060A16AA06988420DD02046FFF7D0FF0A
:1010C000E06820F4405040F01000E060A06AA061A9
:1010D0002069E062606044F24001E0688843E060BB
:1010E00010BD000010000200002801D000F024B85C
:1010F0007047000010B5014602A000F065F801201D
:1011000010BD000053494752545245443A2052659D
:101110006469726563743A2063616E2774206F702E
:10112000656E3A200000000010B500F067F8BDE8D9
:101130001040FFF7D9BF000001491820ABBEFEE701
:101140002600020000210160C0E901107047102054
:101150007047034640688C46002818BF88423CBF51
:1011600003464068F8D318681844884207D00CF149
:10117000030020F00700001D411A521A0146081D05
:101180000A60FFF75FBC10B50146C268900703D044
:10119000900607D5886A0AE0FFF788FA0121016006
:1011A000881E10BD8B69486818440B69C01A91F8F5
:1011B00048301BB191F84910401A10BD1103FCD5FD
:1011C0000028FADD401E10BD70B505460C460A2009
:1011D00000E06D1C00F03AF835B128780028F8D10D
:1011E00002E0641C00F032F814B120780028F8D135
:1011F000BDE870400A2000F029B8000010B50128B1
:1012000005D0002103A0FFF7DFFF012010BD09A1D9
:10121000F8E7000053494752544D454D3A204F7569
:1012200074206F662068656170206D656D6F7279DE
:10123000000000003A2048656170206D656D6F7296
:101240007920636F727275707465640008B56946C1
:101250008DF800000320ABBE08BDFEE738B504469C
:101260000020009063696A460121206898476FF06A
:101270000405002825DB63696A4601212068984738
:1012800000281EDB0098400701D4012038BD6369A7
:101290006A46002120689847002812DB0098C104A4
:1012A00008D44FF4045181431DD081041DD4C005DE
:1012B0001DD416E063696A4610212068984700280B
:1012C00001DA284638BD0098C10501D4062038BD92
:1012D000C0F34101022906D010F0060F05D0032902
:1012E00005D0052038BD022038BD032038BD0420BC
:1012F00038BD2DE9F8430446002006460546009017
:101300006068A8BBA06800B1804720206FF0040788
:10131000206063696A46192130469847002801DA3F
:101320003D4607E0009800F01F00B04202D10025C2
:10133000266002E0761C1F2EEBD920681F2802D9F8
:101340006FF0020530E07DBB23694FF400420021BD
:101350009847002830DB63696A4600212068984777
:10136000002827DBA069804706464FF4FA780CE096
:101370000EE0A0698047801B404518D863696A4623
:10138000002120689847002814DB00980004F0D45E
:10139000A069804706464FF4FA67A0698047801B22
:1013A000B842FAD9012060602846BDE8F8836FF0A2
:1013B0000105F9E73D46F7E76FF00305F4E788B16B
:1013C000CA687AB18A686AB10A695AB10A688260E1
:1013D0004A68C260CA6842618A68026109698161BB
:1013E000002070474FF0FF3070477047F0B5002382
:1013F0001A464FF000454FF48C4600BF016903EBDD
:10140000830401EBC4010A604A608A60CA600A6210
:101410000D604A624E604F6827F000474F6000EB56
:101420008307032BB96406D24FF0280C07690CEB35
:10143000C4043C4400E00469CC605B1C042BDDD395
:10144000C26502668266C26682650169006800F54F
:101450008050C160F0BD38B50446006800F580508A
:10146000816941F480118161206800F580508069B4
:101470000090012000F058FA2068009900F5805093
:10148000816138BD014800F0D1BA0000044C002051
:1014900070B5A4B00024012506468DF828408DF8CB
:1014A00004501494A8038DF8564005908DF8105000
:1014B00002948DF85440C0108DF811508DF81F40E3
:1014C0008DF8204006908DF81E508DF80F4009943D
:1014D0008DF81C4012948DF84C408DF855406946AB
:1014E000304600F05DF98DF881508DF880408DF820
:1014F000824028041B908DF8685080011F908DF861
:1015000070508DF8885040128DF871501E941D90C7
:101510008DF87250239421948DF8895019A9304682
:10152000199400F0DDF824B070BD0020704700F081
:101530007DBE000010B5024800F046FC002010BD42
:10154000044C002013460A4610B50146034800F03B
:10155000D7FB002801D04FF0FF3010BD044C002015
:1015600013460A4610B50146034800F03BFD00282B
:1015700001D04FF0FF3010BD044C00202DE9F043A6
:10158000836A1830914650F823208D681C461768EE
:101590000026002F6FDB00EB83077F69C7BBD5F800
:1015A00000C00127C2F808C0D2F804C0D5F80480F2
:1015B0006FF30C0C4CEA080CC2F804C091F800C0A0
:1015C0005FEACC7C09D0D2F800C0D1F814802CF4AA
:1015D000400C4CEA080CC2F800C091F800C05FEA69
:1015E0008C6C09D5D2F800C0D1F810802CF0406C7A
:1015F0004CEA080CC2F800C00978490703D5116805
:1016000041F080011160116841F08051116042E0A9
:1016100031E0116821F0005111601168B9F1000F3B
:1016200002D041F0804101E021F0804111605B1C5B
:10163000042B00D31B1F50F82320116821F0805188
:1016400011601168002903DB00EB83014969A9B12E
:1016500050F8242000210CE0BFF35F8F136823F0C3
:1016600000431360641C042C00D3241F491C50F851
:101670002420B942F0D30220BDE8F083AD68296888
:1016800091605168D5F804C06FF30C0141EA0C0178
:101690005160761C7F1CBFF35F8F116841F00041E1
:1016A0001160A9680029B4D11168B9F1000F02D006
:1016B00041F0804101E021F080411160116841F06A
:1016C0000051116000EB8302416A5161036172B6FF
:1016D000761C816A3144816262B60020CCE700004A
:1016E00070B50C460168054601F5805188692B4AA2
:1016F0001040227BEAB30022637B920642EA4362F7
:10170000637FBBB35FF0000342EA0352A37B42EA6C
:10171000435263691A43237F42EAC312A37F42EA1A
:101720008312236A1A4394F8243042EA8302024364
:101730008A61286800F580508669012000F0F4F87D
:10174000286800F580508661A169A0682279084365
:10175000216941EA4261084394F8251040EAC1102A
:10176000A16A40EA81002168084340F4000128682A
:1017700001E00FE010E000F580500160286800F5FE
:1017800080500468012000F0CFF8286800F58050F0
:10179000046070BD0122AFE70123B5E7233FDEF807
:1017A00070B5026805460C4610683A49237C08402B
:1017B000A168002B63D0002341EAC351637C002B56
:1017C0005FD00023E67F9B0543EA06431943636924
:1017D0001943A37FF3B3002341EA4331237F41EA56
:1017E0000331A3691943237941EA832194F8203016
:1017F0008BB3002341EA4321E37B41EAC311636ACF
:10180000194394F8283041EA031101431160286814
:101810000668012000F088F8286806602A68906948
:101820004FF641710840A36C216D41EA034194F8E1
:101830004C3063B3002394F85560DB01012E00D0D7
:10184000002643EAC603194394F85630012B00D012
:10185000002301E017E018E041EA830194F85430D6
:10186000012B00D0002341EA430101439161286824
:101870008469012000F058F82868846170BD012354
:101880009AE701239EE70123A6E70123B2E701239C
:10189000D1E700000F8120FF2DE9F8434FF0000948
:1018A000CDF80090856E044600EB85004FF00108EE
:1018B000866CE76E1EE0306A30B9684600F052FA76
:1018C000009838B33062B060B8F1000F12D0A06D4C
:1018D00018B34FF48C407060BFF35F8F306840F0F6
:1018E000004030606D1C042D00D32D1F04EB8500DB
:1018F0007F1E866C17B1B8F1000FDCD1E06EB842E4
:1019000006D0206800F58050C0F80890C4E91A5746
:10191000BDE8F8834FF00008ECE70148DBE7000082
:101920000046008072B6FEE770B5044600F07EFC0B
:101930000546601C02D004480078044400F076FCA0
:10194000401BA042FAD370BD380000207047002928
:101950006AD002681268C2F3001281F82820026877
:10196000126802F060024A620268126842F3402282
:10197000521C81F8202002681268C2F30042CA7724
:101980000268126842F34032521C8A770268126879
:10199000C2F300320A770268126802F400628A61B8
:1019A0000268126802F480424A610268126842F3D7
:1019B0008052521C4A740268126842F3C052521C90
:1019C0000A7402681268C2F3C012CA73026812680D
:1019D00002F460228A6002681268C2F380220A71EF
:1019E00002689269C2F3400281F854200268926949
:1019F00042F3C012521C81F84C200268926902F036
:101A000030020A6502689269120C8A64026892695F
:101A1000C2F3800281F8562000688069C0F3C000DC
:101A200081F85500002070470120704710B504462A
:101A3000006800F580504169490607D5C16949062B
:101A400004D52B494161204600F0B0F9206800F52B
:101A500080504169C90708D0C169C90705D04FF056
:101A600001114161204600F0BAFA206800F580506B
:101A70004169090422D5C16909041FD5D4F8881029
:101A800041F00801C4F88810416989040CD5416906
:101A9000184A1140C4F88C10C16921F4C031C161E9
:101AA000E020C4F8840006E0426948F280610A4000
:101AB000C4F88C2041612046FFF748FF2068816B05
:101AC00009070AD5C06A00F06000C4F894002046F7
:101AD00000F014F90020C4F89400074801680903D5
:101AE00005D54FF400210160204600F079FA10BDC1
:101AF0004000010000207E00143C0140F8B50400C5
:101B000003D0D4F8840010B107E00120F8BD2320F1
:101B1000C4F88400204600F07DF83B4800250168A9
:101B200041F480410160006800F480400090374833
:101B3000016821F4000101600168A268114301609D
:101B40000068206800F58050016841F001010160E3
:101B500000F06CFB06464FF4FA770BE000F066FBF2
:101B6000801BB84206D90420C4F88800E020C4F8DD
:101B70008400CAE7206800F580500068C007EDD1F6
:101B80002046FFF785FC0021E06801EB810200EBB5
:101B9000C200056045608560C56004EB8103986103
:101BA000036843F480130360032905D22826E36801
:101BB00006EBC2021A4400E0E268C260026842F426
:101BC00040020260491C0429DED3A5622068E16856
:101BD00000F5805001612046FFF708FC60680C4A60
:101BE000818811640178C37841EA03618378407881
:101BF0001B0443EA002001435164C4F888501020BC
:101C0000C4F884000020F8BD443802400438014084
:101C100000800240F0B587B0044614216846FEF704
:101C20001BFD3149206888425BD13048002401689F
:101C300041F000710160016801F0007105910168D7
:101C400041F080610160016801F0806105910168E7
:101C500041F000610160016801F0006105910168D7
:101C600041F004010160016801F00401059101687F
:101C700041F001010160016801F001010591016875
:101C800041F0020101600068022500F002000590A9
:101C90003220CDE9000502AA03260B2782E8D000F6
:101CA0006946134800F0CAF98620CDE9000502AA6A
:101CB000694682E8D0000F4800F0C0F94FF4605048
:101CC000CDE9000502AA694682E8D0000A4800F082
:101CD000B5F9002211463D2000F042FB3D2000F006
:101CE00031FB07B0F0BD00000080024030380240F8
:101CF000000802400000024000040240704700005B
:101D00002DE9F041984603680546186900F01C0467
:101D10004FF6FF7000EAC1204FF4F861204301EA5A
:101D20008211014321F0020040F001041C6100F027
:101D30007DFA06464FF480370AE000BF00F076FADD
:101D4000801BB84202D30120BDE8F08128680469F5
:101D5000E007F3D12868406981B20020C8F800107C
:101D6000F2E700001CB504460D4803F071FE0300C5
:101D70000FD003F1200020600A4818614FF4C061C1
:101D80002068CDE9000100214122084604F0FAFB59
:101D90001CBD054901200870002020601CBD00000A
:101DA000E0C00008E96B000800000020704710B593
:101DB00019B1D0F88420102A01D0012010BDFFF7FE
:101DC000EFFC002010BD000070B5054600680069FA
:101DD00020F01C0400F0B0FB1049114A014491426C
:101DE00002D244F0080416E00E490F4A0144914221
:101DF00002D244F00C040EE00C490D4A0144914219
:101E000009D30C4908440C49884202D244F0040426
:101E100001E044F010042868046170BD00D3CEFED8
:101E2000C0E1E40040F1E9FD40787D0100796CFCFF
:101E3000005A6202001F0AFA80F0FA0270B50446E6
:101E4000D0F88400102801D0012070BD2325C4F8EB
:101E500084500420E0662046FFF71EFD20680168DC
:101E600041F008010160206806680120FFF75CFD71
:101E7000206806602068016841F004010160206864
:101E800006680120FFF750FD206806602046FFF736
:101E9000E2FA206800F58050816941F400518161C7
:101EA000206800F58050816941F002018161C4F829
:101EB0008450002070BD70B50446D0F884002328FB
:101EC00001D0012070BD2320C4F88400206800F5F3
:101ED0008050816921F400518161206800F58050B3
:101EE000816921F0020181612068016821F004010B
:101EF0000160206805680120FFF716FD2068056075
:101F00002046FFF7A8FA2068016821F00801016067
:101F1000206805680120FFF707FD20680560102094
:101F2000C4F88400002070BD2DE9F0411546044638
:101F300021B1D4F88400232805D04EE054F8880F4E
:101F400040F0010008E000222046FFF717FB28B10F
:101F500054F8880F40F0020020603EE0BFF34F8F3E
:101F6000A06A04EB8001401C8E69A062042801D3A2
:101F7000001FA06204EB80008169206800F580509A
:101F8000416000F053F9074619E0206800F58050E1
:101F9000406980040BD554F8880F40F00800206099
:101FA00054F8880C00F580504069606015E0681CAA
:101FB00005D000F03BF9C01BA84206D82DB130680F
:101FC0000028E2DB0020BDE8F08154F8880F40F0E3
:101FD000040020604FF0405030600120F3E770476C
:101FE000704700002DE9F04106680546306900F0B1
:101FF0001C044FF6FF7000EAC1204FF4F861204343
:1020000001EA8211014398B241F00304706128682B
:10201000046100F00BF906464FF480370AE000BF78
:1020200000F004F9801BB84202D30120BDE8F08122
:1020300028680469E007F3D1F8E700002DE9F84FBC
:10204000DFF8BCA10022012503264FF00F090AF199
:10205000040BAAF1040E00BF0B6805FA02F423403A
:10206000A34270D10F7907F00307012F01D0022F8F
:1020700016D187684FEA420806FA08FC27EA0C07DF
:10208000D1F80CC00CFA08FC4CEA070CC0F808C0E8
:102090004768A7430C79C4F3001494403C43446060
:1020A0000C79E443A4070AD0C4684FEA420C06FA4C
:1020B0000CF7BC438F6807FA0CF72743C7600C790D
:1020C00004F00304022C12D1D40800EB840CDCF8D9
:1020D00020405707FF0E09FA07F824EA0804D1F850
:1020E000108008FA07F848EA0408CCF82080046851
:1020F0004FEA420C06FA0CF7BC430F7907F00307CE
:1021000007FA0CF7274307604C6814F4403F70D07F
:102110003C4C276847F480472760246822F0030777
:1021200004F480440094384C07EB040CDCF80848B5
:1021300097074FEA177809FA08F7BC43334FB842BC
:1021400002D1002724E054E0314FB84201D10127E9
:102150001EE0304FB84201D1022719E02E4FB8429D
:1021600001D1032714E02D4FB84201D104270FE01D
:102170002B4FB84201D105270AE02A4FB84201D1BE
:10218000062705E0284FB84201D1072700E00827BD
:1021900007FA08F72743CCF80878DAF800405746E2
:1021A000D1F804C09C435FEACC2C00D51C433C60B2
:1021B000DBF800405F46D1F804C09C435FEA8C2CFA
:1021C00000D51C433C60DEF800407746D1F804C0DF
:1021D0009C435FEA8C3C00D51C433C60084F083FA1
:1021E0003C68D1F804C09C435FEACC3C00D51C435A
:1021F0003C60521C102AFFF42FAFBDE8F88F00009E
:10220000083C0140443802400030014000000240D8
:102210000004024000080240000C0240001002408E
:102220000014024000180240001C0240014880686F
:10223000704700003800002002488168027811448D
:1022400081607047380000200B4810B5016841F4E8
:1022500000710160016841F480610160016841F42E
:1022600080710160032000F09BF80F2000F006F859
:1022700000F050F8002010BD003C024030B505468B
:102280001F4887B00024016841F004010160006824
:1022900006A900F00400009001A800F02DF90498B0
:1022A000A8B100F04FF940001649174AB0FBF1F110
:1022B0001648491E026040F2E732C0E90324C0E933
:1022C0000114846100F038FB040003D015E000F035
:1022D00039F9E9E70D4800F05DFB04000DD11E203F
:1022E00000F030F8102D07D2002229461E2000F001
:1022F00037F80748056000E0012407B0204630BDEC
:102300004038024040420F0000080040F800002022
:102310003C0000200A4808B5016841F48041016092
:10232000006800F4804000900548001F016841F0FB
:1023300080510160006800F08050009008BD0000EE
:1023400044380240002809DB00F01F0201219140BF
:102350004009800000F1E020C0F800117047000043
:10236000F0B40E4B1B680C46C3F30223C3F1070500
:10237000042D00D90425191D072901D2002300E0EE
:10238000DB1E012606FA05F1491E214099409E40B8
:10239000761E16403143F0BC00F085BD0CED00E028
:1023A000064900F0070208684FF6FF03184040EAAC
:1023B0000220034A10430860704700000CED00E063
:1023C0000000FA052DE9F0470E46050065D0DFF85C
:1023D0001481D8F80000F7B200F00700B04207D22D
:1023E00088F80070D8F8000000F00700B04254D11F
:1023F00028683D4C810712D5400703D5206840F47A
:10240000E05020602878000703D5206840F4604041
:1024100020602068A96820F0F00008432060287838
:10242000C0072DD0304968680839012812D0022829
:1024300013D0032811D00968890700292DDA2168F3
:1024400021F0030101432160FFF7F0FE814641F2D4
:10245000883A0EE009688903EFE709688901ECE72B
:10246000FFF7E4FEA0EB0901514502D90320BDE8C6
:10247000F0872068696800F00C00B0EB810FEFD1A5
:10248000D8F80010404601F00701B14207D90770A3
:10249000006800F00700B04201D00120E7E728788B
:1024A000400705D52068E96820F4E0500843206023
:1024B0002878000706D52068296920F4604040EAA2
:1024C000C100206000F04EF82168084AC1F30311F2
:1024D000515CC8400649086006480068FFF7CEFE18
:1024E0000020C4E7003C024008380240ECC000086D
:1024F000440000203C0000200F2202600C4A1368B8
:1025000003F003034360136803F0F0038360136870
:1025100003F4E053C36012684FF4E05303EAD202BD
:1025200002610448006800F007000860704700007E
:1025300008380240003C0240014800687047000033
:10254000440000200448054900680968044AC1F3B2
:102550008221515CC8407047440000200838024086
:10256000FCC00008154810B5006810F00C021448B3
:1025700013D01449042A0FD0082A0ED10F4C241F5F
:102580002268236802F03F025B0207D52068C0F38F
:102590008810A0FB010106E0084610BD2168C1F3C8
:1025A0008811A1FB00010023FDF78AFE2168C1F319
:1025B0000141491C4900B0FBF1F010BD0838024050
:1025C0000024F40040787D012DE9F84F04006ED01E
:1025D0002078DFF84C93C007A9F104054AD009F12F
:1025E00004000168C1F38101012908D00068C0F32B
:1025F000810002280AD1D9F80000400206D52868D7
:10260000800337D560680028E1D033E06068B0F51A
:10261000803F10D0B0F5A02F286810D020F4803073
:102620002860286820F4802028606068A8B1FFF73F
:10263000FDFD06460DE0286840F48030F4E740F4E4
:1026400080202860F7E700BFFFF7F0FD801B6428BB
:1026500073D828688003F7D50CE0FFF7E7FD06463E
:1026600005E000BFFFF7E2FD801B6428F0D8286872
:102670008003F7D42078DFF8AC8280074FF0000A9F
:102680003ED5A748001D016811F00C0F08D0006866
:10269000C0F3810002280BD1D9F80000400207D412
:1026A0002868800716D5E068012800D112E033E1E0
:1026B000E068B8B10120C8F80000FFF7B7FD064692
:1026C00005E000BFFFF7B2FD801B0228C0D82868D4
:1026D0008007F7D52868216920F0F80040EAC1009A
:1026E00028600DE0C8F800A0FFF7A0FD064604E052
:1026F000FFF79CFD801B02281FD828688007F7D4AD
:102700002078000722D5864F87486169703771B1FC
:1027100001210160FFF78AFD064604E0FFF786FD10
:10272000801B022809D838688007F7D50EE0C0F86A
:1027300000A0FFF77BFD064605E082E0FFF776FD8F
:10274000801B02287DD838688007F7D4207840079E
:1027500068D5DFF8CCB100270BF13C0BDBF80000AB
:10276000C0000BD4DBF8001041F08051CBF8001012
:10277000DBF80000012700F0805000906B4E3068BD
:10278000C00510D4306840F480703060FFF74EFD13
:10279000009005E0FFF74AFD0099401A022850D842
:1027A0003068C005F6D55E4EA0686C3601280FD0A3
:1027B0000528306810D020F001003060306820F02B
:1027C00004003060A068B8B1FFF730FD00900FE062
:1027D000306840F00100F4E740F004003060F7E7B3
:1027E000FFF724FD0099411A41F28830814266D8F2
:1027F00030688007F4D50EE0FFF718FD009007E081
:10280000FFF714FD0099411A41F28830814256D8F1
:1028100030688007F4D42FB1DBF8001021F080512C
:10282000CBF80010A069C8B33D49091D0968C1F380
:10283000810102294AD00228504607D0C8F860001A
:1028400000E03CE0FFF7F2FC04463BE04746C8F8F6
:102850006000FFF7EBFC064605E000BFFFF7E6FC73
:10286000801B02282BD828688001F7D4D4E90701FF
:102870000843A16A2E4A490802EB0141626A41EA13
:102880008211084394F82C1040EA0161C9F8001045
:1028900001203866FFF7CAFC044606E03EE000BFB0
:1028A000FFF7C4FC001B022809D828688001F7D56F
:1028B00034E000BFFFF7BAFC001B022802D9032056
:1028C000BDE8F88F28688001F4D427E00128F7D00C
:1028D000D9F80000E26900F4800191421CD1226A1B
:1028E00000F03F01914217D147F6C071626A014082
:1028F000B1EB821F10D1A26A4FF0FF3300F44031D8
:1029000003EB5202B1EB024F06D194F82C1000F009
:102910007060B0EB016F01D00120D1E70020CFE75C
:102920000438024000004742800E474200700040D9
:102930000000FFFF7047704710B5040003D094F803
:102940003D0010B107E0012010BD002084F83C00DC
:10295000204600F01EF8022084F83D00211D20686A
:1029600000F03CFA012084F8460084F83E0084F828
:102970003F0084F8400084F8410084F8420084F865
:10298000430084F8440084F8450084F83D000020AA
:1029900010BD704790F83D10012901D0012070470B
:1029A000022180F83D100168CA6842F00102CA6045
:1029B00000681149884214D0B0F1804F11D00F49FE
:1029C00088420ED00E4988420BD00E49884208D06A
:1029D0000D49884205D00D49884202D00C498842F1
:1029E00004D1816801F00701062903D0016841F094
:1029F0000101016000207047000001400004004018
:102A000000080040000C004000040140004001406C
:102A100000180040704770B50446006801694FF027
:102A20000005C943890715D4C168C943890711D472
:102A3000E91E016101202077206880698007204617
:102A400002D0FFF7E7FF04E000F098F8204600F01E
:102A500096F8257720680169C943490717D4C168EA
:102A6000C943490713D46FF00401016102202077A4
:102A70002068806910F4407F204602D0FFF7CAFF2B
:102A800004E000F07BF8204600F079F82577206814
:102A90000169C943090716D4C168C943090712D49B
:102AA0006FF008010161042020772068C069800769
:102AB000204602D0FFF7AEFF04E000F05FF82046AA
:102AC00000F05DF8257720680169C943C90617D46D
:102AD000C168C943C90613D46FF010010161082011
:102AE00020772068C06910F4407F204602D0FFF7AD
:102AF00091FF04E000F042F8204600F040F825770E
:102B000020680169C943C90708D1C168C943C90719
:102B100004D1891E0161204600F032F82068016965
:102B2000C943090609D4C168C943090605D46FF031
:102B3000800101612046FFF7FDFE20680169C9435D
:102B4000490609D4C168C943490605D46FF040015C
:102B50000161204600F01EF820680169C94389061A
:102B60000BD4C168C943890607D46FF02001016105
:102B70002046BDE87040FFF7DEBE70BD704770476D
:102B800000680349884201D1FFF756BB7047000037
:102B9000000800407047FEE7114808B5016841F0A1
:102BA00080010160016801F080010091016841F03D
:102BB00004010160016801F004010091016841F025
:102BC00001010160016801F001010091016841F01B
:102BD00002010160006800F00200009008BD0000E2
:102BE00030380240FEB5494CC020251D2070A82079
:102BF00060700120A0706F20E070FF202870687066
:102C0000A87000272E1DEF7037707770B770F770BF
:102C100002F008FB208841BA0A04A17842EA0123A5
:102C2000E27844BA2404134344EA01241B06A4B204
:102C300043EA042344BA40BA000440EA0120E4B263
:102C400043EA04231043A5F1100143EA1060086031
:102C5000288841BA0A04A97844BA42EA0123EA78EA
:102C60002404134344EA01241B06A4B243EA0423C8
:102C700044BA40BA000440EA0120E4B243EA042323
:102C80001043A5F10C0143EA10600860308841BA96
:102C90000A04B17844BA42EA0123F27824041343C7
:102CA00044EA01241B06A4B243EA042344BA40BA0E
:102CB000000440EA0120E4B243EA0423104343EA5B
:102CC0001060A5F10801A5F108030860104811493A
:102CD0000097CDE901101A1F111F0F4802F0FEFEE8
:102CE0000D4803F015F90C4890F82D0040070A48EC
:102CF00002D503F021FA01E003F010F903B007490F
:102D0000BDE8F040044803F05DB900002C0000204D
:102D1000813B0008B53D00080C4D0020B93C00087F
:102D2000FEE7FEE7704770477047000030B593B08C
:102D300030216846FDF790FC14210CA8FDF78CFCAF
:102D40001D480025016841F080510160006800F0D5
:102D5000805011901948016841F480410160006879
:102D6000022400F480401190012003901020049070
:102D7000009406940820CDE90750A820CDE9090465
:102D800004200B906846FFF71FFC08B172B6FEE7FF
:102D90000CA90F2081E831004FF4A0500F904FF4A0
:102DA0008050109005210CA8FFF70CFB002801D0E3
:102DB00072B6FEE713B030BD4038024000700040EC
:102DC0000248016841F470010160704788ED00E03D
:102DD0000148FFF720BE0000F8000020F0B50268AF
:102DE000254C264D264E274F274B4FF0804CA042B6
:102DF00009D0604507D0A84205D0B04203D0B84200
:102E000001D0984204D122F0700E4A6842EA0E02C4
:102E1000A0421BD0604519D0A84217D0B04215D0AF
:102E2000B84213D0984211D0184DA8420ED0184D78
:102E3000A8420BD0174DA84208D0174DA84205D084
:102E4000164DA84202D0164DA84203D122F4407577
:102E5000CA682A434D6922F080022A4302608A68C8
:102E6000C2620A688262A04201D0984201D1096917
:102E7000016301214161F0BD0000014000040040F8
:102E800000080040000C00400004014000400140E8
:102E9000004401400048014000180040001C004070
:102EA00000200040FEE70907090E002804DB00F1BE
:102EB000E02080F80014704700F00F0000F1E020DF
:102EC00080F8141D7047000070B505460C46880751
:102ED00006D006A34FF4B67210A118A0FDF768FA49
:102EE000A86800682060A868046070BD2E2E2F4D71
:102EF0006964646C6577617265732F546869726484
:102F00005F50617274792F4C7749502F7372632F21
:102F1000636F72652F6D656D702E63006D656D70EA
:102F20005F667265653A206D656D2070726F7065C1
:102F3000726C7920616C69676E65640041737365BA
:102F40007274696F6E2022257322206661696C6538
:102F500064206174206C696E6520256420696E2090
:102F600025730A0010B580680468002C0CD0216815
:102F70000160A00706D005A34FF48C720FA118A022
:102F8000FDF716FA204610BD002010BD2E2E2F4D45
:102F90006964646C6577617265732F5468697264E3
:102FA0005F50617274792F4C7749502F7372632F81
:102FB000636F72652F6D656D702E63006D656D704A
:102FC0005F6D616C6C6F633A206D656D702070721F
:102FD0006F7065726C7920616C69676E6564000062
:102FE000417373657274696F6E20222573222066A7
:102FF00061696C6564206174206C696E652025646C
:1030000020696E2025730A0070B5094D064600241C
:1030100004EB440005EBC000017D29B18068B0429B
:1030200002D1204600F036F9641C0A2CF0DB70BD9A
:103030007C8200202DE9F74F84B04FF00A0B00246A
:103040000646DA465F46D94602940194CDF8004020
:10305000514904EB440001EBC008039098F8145068
:103060000A2F1DD0002D2AD0012D08D0022D06D206
:103070004AA340F2231257A166A0FDF799F99EB129
:103080003168D8F8040081420ED1069820B1D8F8F2
:1030900008100698814207D1204607B0BDE8F08F9E
:1030A000002DE1D127460AE0012D16D0022D06D3CE
:1030B000B8F812000099884201D3A2460090641C1F
:1030C00024B20A2CC4DB059881074FF0FF30E4D40A
:1030D0000A2F16D018DA3C463EE02F49039851F8E3
:1030E00030000028B8F8120005D002998842E6D3D3
:1030F000A1460290E3E701998842E0D3A3460190FC
:10310000DDE70599C907C8D05146BAF10A0F0EDAB2
:103110000C46214801EB440150F8310080B11FA357
:1031200040F26D1245A13BA0FDF742F908E0594677
:10313000BBF10A0F03DB4946B9F10A0FADDA0C46C1
:103140000A2C06DB15A340F27F1242A131A0FDF745
:103150002FF9204600F09EF80A2C06DB0FA340F260
:1031600083123CA12BA0FDF723F90B4804EB44018B
:1031700000EBC105287D30B108A34FF4C2723AA11B
:1031800024A0FDF715F90EB1306868600020688250
:103190000698A86080E700007C8200202E2E2F4D2C
:1031A0006964646C6577617265732F5468697264D1
:1031B0005F50617274792F4C7749502F7372632F6F
:1031C000636F72652F697076342F657468617270F1
:1031D0002E6300007374617465203D3D20455448A2
:1031E0004152505F53544154455F50454E44494EFF
:1031F00047207C7C207374617465203E3D204554DB
:10320000484152505F53544154455F535441424CDE
:1032100045000000417373657274696F6E2022254A
:103220007322206661696C6564206174206C696E2C
:103230006520256420696E2025730A006172705F25
:103240007461626C655B695D2E71203D3D204E5559
:103250004C4C000069203C204152505F5441424C8C
:10326000455F53495A4500006172705F7461626C3A
:10327000655B695D2E7374617465203D3D20455426
:10328000484152505F53544154455F454D50545945
:103290000000000070B5074C00EB4005002654F814
:1032A000350018B103F0F6FB44F8356004EBC500B7
:1032B000067570BD7C8200202DE9F04385B00D00BD
:1032C000074609D07C684FF480782088404539D182
:1032D0002079062836D109E01CA340F28A2229A1D0
:1032E0002CA0FDF765F805B0BDE8F08360790428EF
:1032F00028D16088082825D1D4F80E000490A1694F
:10330000686820B1814202D10126334601E00026DF
:10331000022304F10802914604A9284600F0A2FB0A
:10332000E08840450ED16EB1022204ABCDE90232F5
:10333000291DCDE9001905F1260319464A462846FC
:1033400000F090FA384603F0A5FBCCE72E2E2F4D67
:103350006964646C6577617265732F54686972641F
:103360005F50617274792F4C7749502F7372632FBD
:10337000636F72652F697076342F6574686172703F
:103380002E6300006E6574696620213D204E554C09
:103390004C000000417373657274696F6E202225C2
:1033A0007322206661696C6564206174206C696EAB
:1033B0006520256420696E2025730A00FEB5154638
:1033C0000E46040006D143A340F21E324FA153A083
:1033D000FCF7EEFF36B93FA340F21F3259A14FA0D0
:1033E000FCF7E6FF35B93BA34FF4487258A14BA058
:1033F000FCF7DEFF2146286800F0B6FE08B1584B06
:103400003FE02868C0F303110E2925D0A168636846
:1034100000EA01020B409A4208D080B2A0F57E413A
:10342000A93903D0E068B0B304F10C054D4B4E4808
:103430001A7802EB420100EBC1010F7D022F2ED35F
:103440008F68A7422BD12F6849688F4227D1314618
:10345000204600F08BF8FEBD01208DF8040000200E
:103460008DF805005E208DF80600687801AB00F04D
:103470007F008DF80700A8788DF80800E8788DF8AF
:1034800009004FF40060009004F126023146204606
:1034900000F014FCFEBDFFE76FF00300FAE7002226
:1034A00002EB420100EBC1010F7D022F08D38F68B0
:1034B000A74205D12F6849688F4201D11A70C6E72B
:1034C000521CD2B20A2AEBD332462946204600F0DB
:1034D000D5F8DFE72E2E2F4D6964646C6577617235
:1034E00065732F54686972645F50617274792F4CF0
:1034F0007749502F7372632F636F72652F697076EF
:10350000342F6574686172702E6300006E65746993
:103510006620213D204E554C4C00000041737365E0
:103520007274696F6E2022257322206661696C6552
:1035300064206174206C696E6520256420696E20AA
:1035400025730A007120213D204E554C4C0000008F
:1035500069706164647220213D204E554C4C00001E
:1035600004C10008E00000207C8200202DE9F8431F
:103570000646154688461C4802EB450100EBC1048F
:10358000207D022806D219A340F2EE2225A131A007
:10359000FCF70EFF144A05EB4501207D02EBC10547
:1035A0000C35022813D1608A0327B0F58E7F04D929
:1035B000211D304600F010FA07E0B0F5877F06D3F2
:1035C0002A46211D304600F00DFA00B927754FF448
:1035D000006000902B4606F126024146304600F07E
:1035E0006DFBBDE8F88300007C8200202E2E2F4D5D
:1035F0006964646C6577617265732F54686972647D
:103600005F50617274792F4C7749502F7372632F1A
:10361000636F72652F697076342F6574686172709C
:103620002E6300006172705F7461626C655B617231
:10363000705F6964785D2E7374617465203E3D200F
:103640004554484152505F53544154455F5354418F
:10365000424C4500417373657274696F6E20222578
:103660007322206661696C6564206174206C696EE8
:103670006520256420696E2025730A002DE9FC5F12
:103680008246263001900E46086814464FF0FF37F8
:103690004FF0000B514600F067FD80B93068C0F371
:1036A00003110E290BD056B148B1524601213046C4
:1036B000FFF7C0FC050005D540B2BDE8FC9F6FF0E8
:1036C0000F00FAE77F2D06D337A340F2C13244A1A1
:1036D00047A0FCF76DFE05F0FF094F4909EB4908CB
:1036E00001EBC805287D00280ED0012808D002284B
:1036F00006D22DA340F2CD3248A13DA0FCF758FEE2
:10370000BBF1000F06D104E001202875C5F808A020
:1037100000E034B93146504600F05EF90746002C0F
:10372000CBD0287D3C4E02280ED346494FF4006092
:1037300005F10C0381F80090009021465046019A53
:1037400000F0BCFA07462DE001282BD1254640F2B7
:10375000F13768892989884207D1286828B112A3DE
:103760003A4639A122A0FCF723FE287B400607D564
:1037700022464FF420710E2002F0C2FF044605E0FD
:103780002D68002DE5D1204603F0F0FA44B156F83B
:10379000380008B103F07EF946F83840002701E010
:1037A0004FF0FF37384688E72E2E2F4D6964646C42
:1037B0006577617265732F54686972645F506172D6
:1037C00074792F4C7749502F7372632F636F726532
:1037D0002F697076342F6574686172702E630000F3
:1037E00074797065206F766572666C6F7700000083
:1037F000417373657274696F6E202225732220668F
:1038000061696C6564206174206C696E6520256453
:1038100020696E2025730A007C8200206172705F2F
:103820007461626C655B695D2E7374617465203DC3
:103830003D2050454E44494E47206F72205354411D
:10384000424C4500E00000206E6F207061636B65A4
:10385000742071756575657320616C6C6F77656434
:10386000210000002DE9FF4F81B09846DDE90FA946
:10387000DDF838B006004FF0000706D12CA340F267
:10388000574239A13CA0FCF793FD4FF420721C2154
:103890000E2002F005FD050046D068891C2806D2DE
:1038A00023A340F262423EA133A0FCF781FD6C6885
:1038B000119801F0B5FCE08096F82C00062806D09F
:1038C0001BA340F2694243492BA0FCF771FDD8F8D5
:1038D0000010A160B8F80400A081DAF80010C4F864
:1038E0001210BAF80400E082DBF80000C4F80E0001
:1038F000D9F80000A0614FF480702080082060801B
:10390000062020710420607140F60600DDE90223E4
:1039100000902946304600F0D1F9284603F0BAF865
:10392000384605B0BDE8F08F4FF0FF30F9E70000F2
:103930002E2E2F4D6964646C6577617265732F5408
:10394000686972645F50617274792F4C7749502FA7
:103950007372632F636F72652F697076342F65748D
:10396000686172702E6300006E6574696620213D87
:10397000204E554C4C000000417373657274696FA2
:103980006E2022257322206661696C656420617453
:10399000206C696E6520256420696E2025730A00FD
:1039A000636865636B207468617420666972737400
:1039B00020706275662063616E20686F6C6420738E
:1039C0007472756374206574686172705F68647284
:1039D00000000000ECC20008014A00F003B800003B
:1039E00004C100087FB5064D031D0124CDE9003553
:1039F000CDE9021422331946FFF734FF04B070BD3D
:103A00000AC1000870B5164D002400BF04EB440045
:103A100005EBC002117DF1B1508A401C80B250828A
:103A2000B0F5967F0AD2012906D003290AD00429CD
:103A30000AD001290BD00EE0052808D32046FFF755
:103A400029FC08E0042000E00220107503E0111DAD
:103A50009068FFF7C1FF641C0A2CD7DB70BD000023
:103A60007C820020F8B5044690F82C001F461646CC
:103A70000D46062806D020A340F2A9122CA135A09D
:103A8000FCF796FC9DB1286888B1214600F06CFBDC
:103A900068B92878C0F303100E2808D022463946AA
:103AA0002846FFF7C7FA002804DA40B2F8BD6FF0E5
:103AB0000F00F8BD00EB40013048022300EBC102CB
:103AC000137594603368D360B388138200235382E4
:103AD00050F8315075B140F831304FF4006000902B
:103AE000334604F126022946204600F0E7F828462E
:103AF00002F0D0FF0020F8BD2E2E2F4D6964646CBB
:103B00006577617265732F54686972645F50617282
:103B100074792F4C7749502F7372632F636F7265DE
:103B20002F697076342F6574686172702E6300009F
:103B30006E657469662D3E6877616464725F6C655A
:103B40006E203D3D204554485F4857414444525FF4
:103B50004C454E00417373657274696F6E20222567
:103B60007322206661696C6564206174206C696EE3
:103B70006520256420696E2025730A007C82002060
:103B80002DE9F041044640890E270D460E283CD908
:103B9000E07B18B995F83000401CE073606801784C
:103BA0008689CA0714D0012905D006221C49FCF7D2
:103BB000C3FC48B10CE0417851B980785E2807D148
:103BC000607B40F0100002E0607B40F00800607312
:103BD000082E03D0B6F5C16F17D10DE095F82D0072
:103BE000000712D53946204603F006F968B9294680
:103BF000204600F001FC10E095F82D00000704D5E8
:103C00003946204603F0F8F818B1204602F042FF8A
:103C100003E029462046FFF74FFB0020BDE8F08176
:103C200004C1000870B59AB0064664216846FCF7E6
:103C300013FD00252C461F48FDF710FB96F82D10AC
:103C400049070DD5012809DC1A48E838FEF733F991
:103C5000304602F063F9304602F0B8F91AB070BD90
:103C60000128FBDD4FF40061CA00022806D00328BA
:103C700005D0042805D00528F0D103E00C461546F0
:103C800000E00C460B486946E838FDF760FE09483D
:103C9000CDE905546946E838FEF789F80548E83863
:103CA000FEF7CCF8304602F047FA304602F0E4F96D
:103CB000D4E70000EC4C0020704700002DE9F041F3
:103CC00004461F4690460E46069801F0A9FA05469E
:103CD0000E21304602F080FA18B16FF00100BDE805
:103CE000F0817068858139680160B9888180D8F871
:103CF0000020C0F80620B8F80410418194F82C0088
:103D0000062806D006A34FF4997213A11FA0FCF752
:103D10004FFB31462046A269BDE8F0411047000044
:103D20002E2E2F4D6964646C6577617265732F5414
:103D3000686972645F50617274792F4C7749502FB3
:103D40007372632F6E657469662F65746865726E31
:103D500065742E63000000006E657469662D3E6810
:103D600077616464725F6C656E206D757374206238
:103D700065203620666F722065746865726E6574A2
:103D80005F6F757470757421000000004173736576
:103D90007274696F6E2022257322206661696C65DA
:103DA00064206174206C696E6520256420696E2032
:103DB00025730A0010B5040006D10BA34FF4B572A9
:103DC00010A114A0FCF7F4FA732084F82E007420DC
:103DD00084F82F00194860611948A061204601F05D
:103DE00053F9002010BD00002E2E2F4C5749502FA4
:103DF0005461726765742F65746865726E65746965
:103E0000662E63006E6574696620213D204E554C18
:103E10004C000000417373657274696F6E20222537
:103E20007322206661696C6564206174206C696E20
:103E30006520256420696E2025730A00BD330008C3
:103E4000715100088A68002A01DCFCF722BE521E6C
:103E50008A604A68C0B2531C4B60107070470A46B3
:103E6000032100F0F5B800002DE9FE4F8A464449D1
:103E70000446D1F8088098F800000007850E142D3C
:103E800079D36089042876D360680078002872D0DE
:103E9000082870D1486901F11407C0F303120E2AF3
:103EA00069D08946096800F05FF9002863D120894C
:103EB000082860D305F10E010E46204602F08CF969
:103EC000002830D02089411989B2884253D84FF454
:103ED00020720E2002F0E4F906004CD0718905F141
:103EE0000800814216D32A4641467068FCF76FFBF2
:103EF0002946304602F080FF002806D021A3B622D2
:103F00002EA13CA0FCF754FA04E02146304602F012
:103F100045FC18B1304602F0BDFD2CE0204602F011
:103F2000B9FD34460CE03146204602F065FF00281A
:103F300006D014A3C72239A12EA0FCF739FA1AE043
:103F400029462046666802F047F9A0B960683968DA
:103F5000FF22C160D9F81010016100213170718019
:103F60000272418101228DE806040A46FF23394688
:103F7000204600F011FB2046BDE8FE4F02F08ABD4E
:103F8000404D00202E2E2F4D6964646C6577617260
:103F900065732F54686972645F50617274792F4C35
:103FA0007749502F7372632F636F72652F69707634
:103FB000342F69636D702E630000000069636D70BB
:103FC0005F696E7075743A206D6F76696E672072E6
:103FD0002D3E7061796C6F616420746F2069636D30
:103FE0007020686561646572206661696C65640A49
:103FF00000000000417373657274696F6E202225A2
:104000007322206661696C6564206174206C696E3E
:104010006520256420696E2025730A0069636D7030
:104020005F696E7075743A20726573746F72696E31
:1040300067206F726967696E616C20702D3E7061D8
:10404000796C6F6164206661696C65640A000000C8
:104050002DE9FF479146884606464FF420722421F9
:10406000222002F01DF9050031D06889242806D2EB
:1040700018A34FF4B47225A12FA0FCF799F96C682E
:1040800077681C2284F8008084F801904FF00008C3
:10409000A4F80480A4F80680686871680830FCF70A
:1040A00096FAF868039003A800F086FC60B1A4F8C3
:1040B00002800122CDF80080CDE90120FF2303AA70
:1040C0000021284600F068FA284602F0E3FCBDE82B
:1040D000FF8700002E2E2F4D6964646C6577617236
:1040E00065732F54686972645F50617274792F4CE4
:1040F0007749502F7372632F636F72652F697076E3
:10410000342F69636D702E6300000000636865637F
:104110006B207468617420666972737420706275B4
:10412000662063616E20686F6C642069636D702027
:104130006D65737361676500417373657274696F50
:104140006E2022257322206661696C65642061748B
:10415000206C696E6520256420696E2025730A0035
:104160000A460B21FFF774BF421C12D088B191F8A8
:104170002D2092070BD54B68834208D0896800EA4E
:1041800001020B409A4202D10143491C01D0002098
:1041900070470120704700002DE9F74F88B00446B2
:1041A000099800251426808CAF1F1438C11700EB26
:1041B0005170C0F3CF00039060680690017801F061
:1041C0000F01052903D038460BB0BDE8F08F618997
:1041D000142907D25BA34FF43F7269A16FA0FCF7CB
:1041E000E7F8F0E7C08801F01BF8C0F30C0100F419
:1041F000005002910790208914381FFA80F88EE051
:1042000003984FF6FF7101EAC0004146404500D9CE
:10421000084604904FF4207214210E2002F040F85A
:104220005FEA000A7ED0BAF80A00142806D245A335
:104230004FF4497263A159A0FCF7BAF81422DAF8D6
:1042400004000699FCF7C3F9DAF804000590049F0E
:1042500035E06089811B8DB2B04206D239A340F2AD
:104260002D3260A14DA0FCF7A3F8AF4200D23D462D
:104270001DB3052001F09AFB5FEA000957D0606882
:104280004B463044CDE9000541222946002002F08A
:1042900079F95FEA000B50D0204602F067FD5549DE
:1042A000C9E904145946504602F088F9781B0704FE
:1042B0003F0C06D000262468CBE724680026002F98
:1042C000C7D1701986B20998808C1438404502987D
:1042D000C0F30C0001DB079909B140F4005000F075
:1042E0009FFF0599C8800498143080B200F098FFB1
:1042F00005994880059800214181099851460A9AFC
:1043000043699847504602F0C5FB0499A8EB0100A9
:104310001FFA80F8DDE90201084480B20290B8F18A
:10432000000F00E006E07FF46BAF00204CE7504642
:1043300002F0B0FB4FF0FF3046E7484600F06CFB60
:10434000F5E700002E2E2F4D6964646C657761726D
:1043500065732F54686972645F50617274792F4C71
:104360007749502F7372632F636F72652F69707670
:10437000342F6970345F667261672E63000000003D
:104380006970345F6672616728293A2070627566C9
:1043900020746F6F2073686F7274000041737365CF
:1043A0007274696F6E2022257322206661696C65C4
:1043B00064206174206C696E6520256420696E201C
:1043C00025730A0074686973206E656564732061E3
:1043D000207062756620696E206F6E652070696559
:1043E00063652100702D3E6C656E203E3D20706F30
:1043F00066660000F14F00082DE9F0474568074662
:104400000E4628780421B1EB101F03D0384602F085
:1044100041FB77E000074FEA9068688800F000FFF2
:1044200004463889A04203D92146384602F004FCEC
:1044300079894145EAD33889A042E7D3B8F1140F0E
:10444000E4D32969DFF81C91C1F303100E28C9F8E1
:104450001410EA68C9F8102005D0304600F086F83C
:1044600050B1344619E096F82D00C00702D07068AC
:104470000028F6D1002410E099F8140000247F28C9
:104480000BD03948046806E0B44203D0204600F05F
:104490006DF810B92468002CF6D13146D9F8100017
:1044A000FFF762FE0028B1D199F81000C0F30310A5
:1044B0000E28ABD0002CA9D0E88830F0C00005D081
:1044C000384600F035F907001CD07D68C9F808505F
:1044D000C9E90046297838460907890EA9F80C1061
:1044E000414602F089FC687A012818D0062811D0CC
:1044F00011280AD04D462146D9F81400FFF734FEA2
:1045000090B11EE00020BDE8F0873146384607F044
:104510004DFC19E03146384603F028FD14E03146E1
:104520003846FFF7A1FC0FE0287DC0F303100E28EA
:1045300007D04146384602F067FB02213846FFF7B4
:104540008EFC384602F0A6FA0021C9F80010C9F81E
:104550000410C9F80810A9F80C10C9F81010C9F80F
:104560001410CFE7404D00207C00002010B590F8DB
:104570002D10C9070CD0416851B1064A52698A42D0
:1045800004D001461046FFF7EFFD08B1012010BD31
:10459000002010BD404D0020FEB5DDE90954089E05
:1045A0001AB109B10F6807B9211D0096CDE9015470
:1045B00000F002F8FEBD00002DE9F84F0546DDE9E8
:1045C0000BA8807BDDF828B01F46164689460128D7
:1045D00006D02FA34FF455723AA13DA0FBF7E8FE99
:1045E0006FF00104002E35D01421284601F0F4FDAF
:1045F000002832D168896C68142806D224A34FF4AD
:1046000062723DA132A0FBF7D3FE277284F809A0A5
:10461000306820614520207084F801B0288900F0BE
:10462000FFFD414F60804FF0000AA4F806A03888D3
:1046300000F0F6FDA0803888401C3880B9F1000FEA
:1046400005D0D9F80000E060A4F80AA00CE03748D3
:104650000068F8E76889142802D22046BDE8F88F80
:1046600068686E4600690090B8F8240040B1298956
:10467000814205D9324641462846FFF78DFDEDE7D8
:10468000D8F814304046324629469847E6E70000FD
:104690002E2E2F4D6964646C6577617265732F549B
:1046A000686972645F50617274792F4C7749502F3A
:1046B0007372632F636F72652F697076342F697020
:1046C000342E6300702D3E726566203D3D20310022
:1046D000417373657274696F6E20222573222066A0
:1046E00061696C6564206174206C696E6520256465
:1046F00020696E2025730A00636865636B20746807
:1047000061742066697273742070627566206361DB
:104710006E20686F6C6420737472756374206970A6
:104720005F68647200000000E20000200CC2000814
:104730002DE9F05F45688346287800F00F000528D2
:104740007DD1E88800F06CFDC004070C688800F09B
:1047500067FD29780907890E814270D8401A1FFA2F
:1047600080F8584601F0C2FF6A4C06462088304463
:104770000A2809D93146284600F0E4FB00285ED01B
:10478000208830440A28E8D8A14664684FF0000A1F
:104790000CE06069E968884207D1A069296988420C
:1047A00003D1A089A988884203D02468002CF0D1C5
:1047B00006E02CB1E88800F033FDC0041BD025E0F2
:1047C000042001F0F3F804000AD13146284600F035
:1047D000B9FBB04233DB042001F0E8F80400CED08E
:1047E0002021FBF739FF0F20E077D9F80410216072
:1047F000C9F8044004E0E08900F012FDC00405D0CF
:104800001422294604F10800FBF7E1FEA87940F3E1
:1048100040156D1C08D007EB080080B2B84263D386
:104820004FF6EB7188425FD82A465946204600F081
:104830003BF9411C58D0B9F80020324400E064E054
:10484000A9F8002035B107EB0801A183A17F41F051
:104850000101A177012845D1A08B1422143087B221
:10486000606804F10801456828462E68FBF7AFFE32
:10487000384600F0D5FC6880A5F806A0A5F80AA087
:10488000656809E014213046776802F0B5FA3146D0
:10489000284601F093FE3E68002EF3D1D9F80410AB
:1048A0004E468C4205D1002105E00868A04202D0A6
:1048B00001460029F9D1204600F01AFA284601F0F5
:1048C00015FF04463088A04206D213A340F29B2273
:1048D00020A127A0FBF76CFD3088001B3080284604
:1048E000BDE8F09F0020FBE7606870B9D9F80400CC
:1048F000844206D008A340F2AB2227A11CA0FBF7FC
:1049000057FD0021204600F0F3F9584602F0C2F8A6
:10491000E8E70000E40000202E2E2F4D6964646C4F
:104920006577617265732F54686972645F50617254
:1049300074792F4C7749502F7372632F636F7265B0
:104940002F697076342F6970345F667261672E63E9
:104950000000000069705F72656173735F7062755B
:1049600066636F756E74203E3D20636C656E00005B
:10497000417373657274696F6E20222573222066FD
:1049800061696C6564206174206C696E65202564C2
:1049900020696E2025730A006E6F74206669727339
:1049A00074616C74686F756768206A7573742065CC
:1049B0006E7175657565640070B50146144813E045
:1049C00090F82D20D3070FD053070DD543685BB166
:1049D00084680D68234005EA04069E4216D09207BB
:1049E00002D4C268954211D000680028E8D1094875
:1049F000006850B190F82D20D30706D0520704D597
:104A0000426812B109787F2900D1002070BD0000F2
:104A10007C0000208000002010B5040006D106A311
:104A20004FF4317213A116A0FBF7C2FC2146BDE87A
:104A30001040052000F002BF2E2E2F4D6964646CDB
:104A40006577617265732F54686972645F50617233
:104A500074792F4C7749502F7372632F636F72658F
:104A60002F697076342F6970345F667261672E63C8
:104A7000000000007020213D204E554C4C000000ED
:104A8000417373657274696F6E20222573222066EC
:104A900061696C6564206174206C696E65202564B1
:104AA00020696E2025730A002DE9F05F4C680646E8
:104AB00093460F4600254FF00108608800F0B0FBD8
:104AC00021784FF0FF3A0907890E814231D8A0EBD7
:104AD0000109E08800F0A4FBC0047C68010C002000
:104AE000206001EB090083B2A180E3808B4220D3D8
:104AF000726829E05068B0F804C0614515D22260A0
:104B00006DB1B5F806C0614513D38088834210D8D3
:104B10002F60A088844506D04FF0000803E080880D
:104B2000834206D877608AB12EE002D0C2889142D3
:104B300002D25046BDE8F09F25B1EA88624501D017
:104B40004FF0000802680546002AD3D195B1E888E5
:104B5000A188884206D92AA34FF4DB7237A13FA06F
:104B6000FBF726FC2F60E888A18888420CD04FF024
:104B7000000809E0706830B121A34FF4DF7241A151
:104B800036A0FBF715FC7760BBF1000F02D1B07FB8
:104B9000C007CFD0B8F1000F30D07268002A2DD0F6
:104BA00050688088002829D12168204629B14C68A6
:104BB000C088A1888842F7D020E0B8F1000F1DD04E
:104BC00032B90FA340F2DF123CA124A0FBF7F0FBA7
:104BD00070684068A04206D109A34FF4F07237A173
:104BE0001EA0FBF7E5FB206830B105A34FF4F1727E
:104BF00036A11AA0FBF7DCFB01209BE7002099E718
:104C00002E2E2F4D6964646C6577617265732F5425
:104C1000686972645F50617274792F4C7749502FC4
:104C20007372632F636F72652F697076342F6970AA
:104C3000345F667261672E6300000000636865631D
:104C40006B20667261676D656E747320646F6E278A
:104C500074206F7665726C6170000000417373653B
:104C60007274696F6E2022257322206661696C65FB
:104C700064206174206C696E6520256420696E2053
:104C800025730A006E6F2070726576696F757320E8
:104C9000667261676D656E742C2074686973206D2F
:104CA0007573742062652074686520666972737418
:104CB00020667261676D656E7421000073616E69B4
:104CC000747920636865636B0000000076616C692D
:104CD000646174655F646174616772616D3A6E6589
:104CE00078745F70627566213D4E554C4C00000033
:104CF00070B504460C480D464168A14202D12168B6
:104D000041600AE0002D06D108A340F2451216A129
:104D10001CA0FBF74DFB206828602146BDE87040D1
:104D2000042000F08BBD0000E40000202E2E2F4D4B
:104D30006964646C6577617265732F546869726425
:104D40005F50617274792F4C7749502F7372632FC3
:104D5000636F72652F697076342F6970345F667285
:104D600061672E630000000073616E6974792063CF
:104D70006865636B206C696E6B6564206C69737425
:104D800000000000417373657274696F6E20222504
:104D90007322206661696C6564206174206C696EA1
:104DA0006520256420696E2025730A002DE9F047EF
:104DB000054600240F46A94205D12FA3AB223DA1F1
:104DC0003FA0FBF7F5FA002F08D03868A84205D0BD
:104DD00029A3AD2244A13AA0FBF7EAFA6E684FF48A
:104DE00080387068818800291AD1006868601422B0
:104DF00005F108017068FBF7EAFB01213046FFF777
:104E0000AFF9304601F072FC0446404505D31AA3C1
:104E1000BC223AA12AA0FBF7CBFA304601F03AFEB9
:104E20006E6812E07068B1460668484601F05EFCA4
:104E30000444444505D310A3CC2230A120A0FBF7A5
:104E4000B7FAA4B2484601F025FE002EEAD1394651
:104E50002846FFF74DFF314D2888A04205D206A312
:104E6000D2222FA116A0FBF7A3FA2888001B2880C6
:104E70002046BDE8F08700002E2E2F4D6964646C3B
:104E80006577617265732F54686972645F506172EF
:104E900074792F4C7749502F7372632F636F72654B
:104EA0002F697076342F6970345F667261672E6384
:104EB000000000007072657620213D20697072004C
:104EC000417373657274696F6E20222573222066A8
:104ED00061696C6564206174206C696E652025646D
:104EE00020696E2025730A00707265762D3E6E650E
:104EF0007874203D3D206970720000007062756614
:104F0000735F6672656564202B20636C656E203C60
:104F10003D2030786666666600000000E4000020F0
:104F200069705F72656173735F70627566636F75D8
:104F30006E74203E3D2070627566735F66726565B3
:104F4000640000002DE9F0471D4F89460646002405
:104F50000022134611461546786822E0D0F814C0A6
:104F6000D6F80C80C4450BD1D0F818C0D6F8108004
:104F7000C44505D1B0F80CC0B6F80480C44509D0CA
:104F80006D1C2AB190F81FC092F81F80C44501D84B
:104F900002461946D0F800C0BCF1000F00D003460D
:104FA00060460028DAD11AB11046FFF7FFFE04442C
:104FB0004C4501DA012DCBDC2046BDE8F08700002E
:104FC000E400002070B50948002544680BE0E07F4C
:104FD00020B1401EE0772546246804E0204624687E
:104FE0002946FFF7E3FE002CF1D170BDE40000205C
:104FF00010B5040006D108A340F2CE2215A118A0D6
:10500000FBF7D6F9606908B101F044FD2046BDE820
:105010001040FFF701BD00002E2E2F4D6964646C17
:105020006577617265732F54686972645F5061724D
:1050300074792F4C7749502F7372632F636F7265A9
:105040002F697076342F6970345F667261672E63E2
:105050000000000070637220213D204E554C4C0032
:10506000417373657274696F6E2022257322206606
:1050700061696C6564206174206C696E65202564CB
:1050800020696E2025730A002DE9FC41354C054648
:105090003348206000268DF8006080208DF80100E4
:1050A000E1208DF802008DF804608DF803608DF822
:1050B0000560C4F804D04FF40000A060A4F1A00083
:1050C000E060A03820614FF4C06060612046FCF7CA
:1050D00015FD0746382104F1B000FBF7BDFA04F1D5
:1050E000B000212101604FF44001C0E904611E4875
:1050F00000F046FC062085F82C0060681B4900780B
:1051000085F826006068407885F827006068807818
:1051100085F828006068C07885F829006068007903
:1051200085F82A006068407985F82B0040F2DC5051
:10513000A88495F82D0040F00A0085F82D0004F1B0
:10514000E800FCF73CF904F1E800FCF7D2F81FB1E5
:10515000FCF7E8FBBDE8FC812846FEF763FDF9E7B4
:1051600000800240044C0020E0C000080400002041
:10517000F0B58DB00E4600252F4630216846FBF76E
:105180006BFA30216846FBF767FA3446684600221E
:1051900016E0042D03D36FF00B000DB0F0BD05EB4E
:1051A0004501636840F8213000EB810163894B6061
:1051B0000DB141F8041C236803B98A6024686D1C92
:1051C000002CE6D1054932894E63C1E90120142241
:1051D000A1F1B000FCF7A8FE3846DEE7B44C002091
:1051E00010B504464068804701F044FF094A216831
:1051F00052688B181A1AB2F1004F03D308442246A2
:10520000054902E0044922461846BDE8104001F075
:1052100095BF0000CC000020E151000800BA7047A3
:1052200040BA704710B500F0E5F800F099FB00F0C7
:10523000D9FD06F0AFFD02F08DFEBDE8104001F093
:10524000F9BFFDF701F8FDF771FDFDF7A5FCFDF7CE
:10525000C9FCFEE72DE9F04100284DD0810704D0BC
:1052600026A340F2732231A132E0394DA0F10804A7
:1052700029688C4203D36A680C30904204D91FA37A
:1052800040F27F2233A123E02079002825D0601A44
:1052900086B2208801F0E8FE0746608801F0E4FE4F
:1052A00021884FF4C863002299420DD86188994241
:1052B0000AD8B14202D00088B04205D1686887425E
:1052C00010D07888B0420DD00CA340F2952228A1CE
:1052D000BDE8F04133A0FBF76BB808A34FF423728D
:1052E0003AA1F5E72271A868844200D2AC6020465A
:1052F000BDE8F04101F0E8BDBDE8F0812E2E2F4D54
:105300006964646C6577617265732F54686972644F
:105310005F50617274792F4C7749502F7372632FED
:10532000636F72652F6D656D2E6300006D656D5F37
:10533000667265653A2073616E6974792063686589
:10534000636B20616C69676E6D656E7400000000B0
:10535000480000206D656D5F667265653A20696C76
:105360006C6567616C206D656D6F7279000000007F
:105370006D656D5F667265653A20696C6C65676125
:105380006C206D656D6F72793A206E6F6E2D6C6951
:105390006E6B65643A20646F75626C652066726539
:1053A00065000000417373657274696F6E20222579
:1053B0007322206661696C6564206174206C696E7B
:1053C0006520256420696E2025730A006D656D5F78
:1053D000667265653A20696C6C6567616C206D6505
:1053E0006D6F72793A20646F75626C6520667265C4
:1053F0006500000070B50B480B4C20F003014FF422
:10540000C86521600D80002048800871284601F0A1
:105410002BFE012160600171058045802068A0603D
:1054200070BD00005B4D0020480000202DE9F047D2
:1054300000286FD0C41C4FF6FC710C404FF4C869B3
:105440000C2C01D20C2401E04C457CD884427AD348
:105450004148C4F5C867824601890288891A8EB21C
:1054600076E0304601F000FE0546007900286CD158
:105470002888801B0838A04267D3288804F11401CB
:10548000801B08384FF0010888421DD330190830BE
:1054900087B24F4506D131A340F287323BA140A0ED
:1054A000FAF786FF384601F0DFFD002101712988F7
:1054B000018046802F8085F804800088484505D00B
:1054C00001F0D2FD478001E085F80480DAF8080099
:1054D0005646854203D014E0008801F0C5FD0179ED
:1054E00011B171688842F7D1B0607168884208D004
:1054F000007930B119A340F2B53233A128A0FAF7F0
:1055000057FF281971680830884208D913A340F260
:10551000B93200E015E033A121A0FAF749FFA8074E
:105520000DD00EA340F2BB323AA11DA0FAF740FF06
:105530000AA340F2BD3243A119A0FAF739FF05F1E1
:105540000800BDE8F08705E0FFE7DAF80000865BB9
:10555000B74286D80020F4E7480000202E2E2F4DB9
:105560006964646C6577617265732F5468697264ED
:105570005F50617274792F4C7749502F7372632F8B
:10558000636F72652F6D656D2E630000696E7661C5
:105590006C6964206E65787420707472000000007D
:1055A000417373657274696F6E20222573222066C1
:1055B00061696C6564206174206C696E6520256486
:1055C00020696E2025730A006D656D5F6D616C6CDE
:1055D0006F633A20216C667265652D3E7573656454
:1055E000000000006D656D5F6D616C6C6F633A204B
:1055F000616C6C6F6361746564206D656D6F727949
:10560000206E6F742061626F76652072616D5F65D8
:105610006E642E006D656D5F6D616C6C6F633A201A
:10562000616C6C6F6361746564206D656D6F727918
:105630002070726F7065726C7920616C69676E653D
:10564000642E00006D656D5F6D616C6C6F633A2058
:1056500073616E69747920636865636B20616C693E
:10566000676E6D656E74000002490988401A80B249
:1056700070470000480000202DE9F05F0646CC1C72
:105680004FF6FC7004404FF4C86A0C2C01D20C2475
:1056900001E054452AD88C4228D33E4F38688642D0
:1056A00002D37868864206D33BA340F2D12246A1BA
:1056B0004BA0FAF77DFE3868864249D379688E425E
:1056C00046D2A6F10805BB46281A87B22888C01B17
:1056D00008381FFA80F94C4506D92FA34FF43972C8
:1056E00049A13FA0FAF764FE4C4503D94FF00000F2
:1056F000BDE8F09F2CD0288801F0B6FC80460079E8
:10570000002827D004F11400484521D83819083062
:1057100084B22888504506D11FA340F2163242A118
:105720002FA0FAF745FE204601F09EFCDBF808208A
:10573000904201D2CBF80800002101712988018034
:1057400047802C800088504502D001F08DFC4480B9
:105750003046CDE72888504506D10FA340F2F52208
:1057600031A11FA0FAF724FE38190830DBF8081021
:10577000B8F8009084B2414504D1204601F074FC91
:10578000CBF80800204601F06FFC00210171A0F861
:105790000090D5E7480000202E2E2F4D6964646CE0
:1057A0006577617265732F54686972645F506172C6
:1057B00074792F4C7749502F7372632F636F726522
:1057C0002F6D656D2E6300006D656D5F7472696D80
:1057D0003A206C6567616C206D656D6F72790000B1
:1057E000417373657274696F6E202225732220667F
:1057F00061696C6564206174206C696E6520256444
:1058000020696E2025730A006D656D5F7472696D85
:105810002063616E206F6E6C7920736872696E6BA5
:10582000206D656D6F727900696E76616C696420B8
:105830006E6578742070747200000000092806D329
:1058400007A34FF4D57212A118A0FAF7B1BD002931
:1058500004D0204A52F82000FDF736BB7047000004
:105860002E2E2F4D6964646C6577617265732F54B9
:10587000686972645F50617274792F4C7749502F58
:105880007372632F636F72652F6D656D702E630089
:105890006D656D705F667265653A2074797065201C
:1058A0003C204D454D505F4D41580000417373659C
:1058B0007274696F6E2022257322206661696C659F
:1058C00064206174206C696E6520256420696E20F7
:1058D00025730A007CC1000818B1002908D0FDF723
:1058E000F3BA04A340F295120EA113A0FAF760BD1B
:1058F000704700002E2E2F4D6964646C65776172CD
:1059000065732F54686972645F50617274792F4CAB
:105910007749502F7372632F636F72652F6D656DBA
:10592000702E6300696E76616C696420706F6F6CB5
:105930002064657363000000417373657274696F5E
:105940006E2022257322206661696C656420617473
:10595000206C696E6520256420696E2025730A001D
:1059600030B5064D002400BF55F8240000F008F8BB
:10597000641CA4B2092CF7D330BD00007CC1000820
:105980008268002111604168C91C21F003010022D6
:1059900007E08368521C1B680B60836819600388EA
:1059A000194443889342F4DC7047000010B509287D
:1059B00008D308A340F2571212A11AA0FAF7F8FC74
:1059C000002010BD214951F82000BDE81040FDF72E
:1059D000C9BA00002E2E2F4D6964646C6577617220
:1059E00065732F54686972645F50617274792F4CCB
:1059F0007749502F7372632F636F72652F6D656DDA
:105A0000702E63006D656D705F6D616C6C6F633AD5
:105A10002074797065203C204D454D505F4D4158B4
:105A200000000000417373657274696F6E20222557
:105A30007322206661696C6564206174206C696EF4
:105A40006520256420696E2025730A007CC100084A
:105A500010B518B1BDE81040FDF784BA04A34FF4A7
:105A60009E720FA113A0FAF7A3FC002010BD000046
:105A70002E2E2F4D6964646C6577617265732F54A7
:105A8000686972645F50617274792F4C7749502F46
:105A90007372632F636F72652F6D656D702E630077
:105AA000696E76616C696420706F6F6C20646573D9
:105AB00063000000417373657274696F6E20222564
:105AC0007322206661696C6564206174206C696E64
:105AD0006520256420696E2025730A002DE9F047B2
:105AE0000400DDE90970089D03D03FB100290DD005
:105AF0000DE035A340F2271240A103E032A34FF49A
:105B0000947245A14DA0FAF753FC1DE0554902B926
:105B1000544A03B9534B00266660A660DFF848C1BB
:105B2000C4F814C0E660A68484F82D60C4E9076553
:105B30004E4D95F800C084F830C02061204600F03A
:105B4000B7F92046B84710B10020BDE8F087B2464B
:105B500040F28B1840F28D1994F83000FF2801D1E3
:105B600084F830A000276E681EE0A64205D116A377
:105B700042463FA131A0FAF71BFC7F1CFF2F05DD39
:105B800011A34A463FA12DA0FAF712FC96F8300067
:105B900094F83010884206D1C8B2401C84F8300016
:105BA000002ED9D102E03668002EDED194F8300004
:105BB000FE2806D0401C28706868206020466C6073
:105BC000C3E785F800A0F7E72E2E2F4D6964646CBB
:105BD0006577617265732F54686972645F50617292
:105BE00074792F4C7749502F7372632F636F7265EE
:105BF0002F6E657469662E63000000006E6574691F
:105C0000665F6164643A20696E76616C6964206ED7
:105C100065746966000000006E657469665F6164A2
:105C2000643A204E6F20696E69742066756E6374E5
:105C3000696F6E20676976656E0000004173736559
:105C40007274696F6E2022257322206661696C650B
:105C500064206174206C696E6520256420696E2063
:105C600025730A000CC20008A95E00087800002015
:105C70006E6574696620616C726561647920616427
:105C800064656400746F6F206D616E79206E657459
:105C90006966732C206D61782E20737570706F7239
:105CA000746564206E756D6265722069732032358B
:105CB0003500000070B50C46054602F0B1FE2146E5
:105CC0002846BDE8704006F0EBB90A68C3689A42FE
:105CD00004D001B90022C260012070470020704743
:105CE000F8B516460C00054606D113A340F2CB12B8
:105CF0001EA122A0FAF75CFB36B90FA34FF4E6729F
:105D00001AA11EA0FAF754FB20686968884211D0D6
:105D100000906868306069463046FFF7CBFF3CB1C1
:105D2000206868600121284600F05EF80120F8BD77
:105D30000020F6E70020F8BD2E2E2F4D6964646C1C
:105D40006577617265732F54686972645F50617220
:105D500074792F4C7749502F7372632F636F72657C
:105D60002F6E657469662E6300000000696E7661AF
:105D70006C696420706F696E74657200417373653D
:105D80007274696F6E2022257322206661696C65CA
:105D900064206174206C696E6520256420696E2022
:105DA00025730A000A6883689A4204D001B9002268
:105DB00082600120704700207047000001000CD075
:105DC0000748406807E000BF90F83020521CD2B26C
:105DD0008A4203D000680028F6D1002070470000F6
:105DE000780000207047000070B50D46040006D111
:105DF0000DA340F26D3219A121A0FAF7D9FA94F857
:105E00002D0041070ED5C1070CD0E9070AD0616803
:105E1000002907D0000705D5211D2046BDE87040A8
:105E2000FDF7DABD70BD00002E2E2F4D6964646C45
:105E30006577617265732F54686972645F5061722F
:105E400074792F4C7749502F7372632F636F72658B
:105E50002F6E657469662E63000000006E657469BC
:105E6000665F69737375655F7265706F7274733A9C
:105E700020696E76616C6964206E657469660000E5
:105E8000417373657274696F6E20222573222066D8
:105E900061696C6564206174206C696E652025649D
:105EA00020696E2025730A006FF00B007047000018
:105EB0002DE9F84F4FF000091D4616460C008246AA
:105EC000C84600D1114C06B9104E05B90F4DACB102
:105ED000206898B100274A4631465046FFF762FFD6
:105EE000424629465046FFF7F0FE002F04D16A468D
:105EF00021465046FFF7F4FEBDE8F88F01276A46B9
:105F000021465046FFF7ECFEE5E700000CC2000812
:105F100001498860704700007800002058B190F86F
:105F20002D10CA070ED001F0FE0180F82D100907D0
:105F300008D5FDF769B804A340F29B320FA117A062
:105F4000FAF736BA704700002E2E2F4D6964646C44
:105F50006577617265732F54686972645F5061720E
:105F600074792F4C7749502F7372632F636F72656A
:105F70002F6E657469662E63000000006E6574699B
:105F8000665F7365745F646F776E3A20696E7661E1
:105F90006C6964206E657469660000004173736506
:105FA0007274696F6E2022257322206661696C65A8
:105FB00064206174206C696E6520256420696E2000
:105FC00025730A00002800D0C161704758B190F8CD
:105FD0002D104A070ED501F0FB0180F82D10C16984
:105FE000002907D0084704A340F206420FA118A0D9
:105FF000FAF7DEB9704700002E2E2F4D6964646CED
:106000006577617265732F54686972645F5061725D
:1060100074792F4C7749502F7372632F636F7265B9
:106020002F6E657469662E63000000006E657469EA
:10603000665F7365745F6C696E6B5F646F776E3AF1
:1060400020696E76616C6964206E65746966000013
:10605000417373657274696F6E2022257322206606
:1060600061696C6564206174206C696E65202564CB
:1060700020696E2025730A0010B5040012D094F830
:106080002D00410717D440F0040084F82D000321AF
:106090002046FFF7A9FEE16900290CD02046BDE8A3
:1060A00010400847BDE8104003A34FF478720FA1D9
:1060B00017A0FAF77DB910BD2E2E2F4D6964646CC0
:1060C0006577617265732F54686972645F5061729D
:1060D00074792F4C7749502F7372632F636F7265F9
:1060E0002F6E657469662E63000000006E6574692A
:1060F000665F7365745F6C696E6B5F75703A20697B
:106100006E76616C6964206E6574696600000000DB
:10611000417373657274696F6E2022257322206645
:1061200061696C6564206174206C696E652025640A
:1061300020696E2025730A0050B190F82D10CA070F
:106140000DD141F0010180F82D100321FFF74CBE65
:1061500003A34FF454720FA115A0FAF729B97047A1
:106160002E2E2F4D6964646C6577617265732F54B0
:10617000686972645F50617274792F4C7749502F4F
:106180007372632F636F72652F6E657469662E6319
:10619000000000006E657469665F7365745F7570FA
:1061A0003A20696E76616C6964206E657469660078
:1061B000417373657274696F6E20222573222066A5
:1061C00061696C6564206174206C696E652025646A
:1061D00020696E2025730A00002200F001B800003B
:1061E00070B5A8B1B1F5803F26D2002918D0048936
:1061F0008BB214FA81F5ADB29D421DD3057B2D06FD
:1062000010D54268511A00F11002914214D30CE0EB
:106210000AA340F2DF1215A117A0FAF7C9F80BE0A4
:10622000002070BD42B14268511A41604189194451
:106230004181E1180181F3E7012070BD2E2E2F4D21
:106240006964646C6577617265732F546869726400
:106250005F50617274792F4C7749502F7372632F9E
:10626000636F72652F706275662E63007020213D2A
:10627000204E554C4C000000417373657274696F79
:106280006E2022257322206661696C65642061742A
:10629000206C696E6520256420696E2025730A00D4
:1062A0002DE9FC5F054690460F461046012A0FD0A7
:1062B00041280DD0B0F5C17F10D0B2F5207F55D068
:1062C00042A340F227124DA153A0FAF771F85CE007
:1062D0000246002000F0FEF8044674E00024A146C7
:1062E0000820FFF763FB060036D005F1030B2BF007
:1062F0000300C0F51470B84200D938468246002029
:10630000CDE900807019133020F0030153463A465E
:10631000304600F083FC3079800706D02BA34FF481
:10632000807247A13CA0FAF743F89421B1EB9B0F90
:1063300006D126A34FF481724DA137A0FAF738F8A1
:1063400094B1C9F80060A7EB0A000704B1463F0CFE
:106350004FF00005C4D136E0524901200870A4B1C5
:10636000204600F097FB10E03446ECE7E81C20F0F4
:106370000301F81C20F00302881880B200F110011C
:1063800089B2824201D88A4202D90020BDE8FC9F2E
:106390000846FFF74BF8041EF8D00020CDE9008036
:1063A0006019133020F003013B461A46204600F0E6
:1063B00035FC2079800706D004A34FF491723AA1EE
:1063C00015A0F9F7F5FF2046E0E700002E2E2F4D2F
:1063D0006964646C6577617265732F54686972646F
:1063E0005F50617274792F4C7749502F7372632F0D
:1063F000636F72652F706275662E630070627566DA
:106400005F616C6C6F633A206572726F6E656F7559
:106410007320747970650000417373657274696FDD
:106420006E2022257322206661696C656420617488
:10643000206C696E6520256420696E2025730A0032
:10644000706275665F616C6C6F633A20706275662E
:1064500020712D3E7061796C6F61642070726F7075
:1064600065726C7920616C69676E6564000000007C
:10647000504255465F504F4F4C5F42554653495A24
:1064800045206D7573742062652062696767657267
:10649000207468616E204D454D5F414C49474E4D1B
:1064A000454E540084000020706275665F616C6C1C
:1064B0006F633A20706275662D3E7061796C6F6112
:1064C000642070726F7065726C7920616C69676EA0
:1064D000656400002DE9FC4114460E460746412A3A
:1064E00008D0012C06D00CA34FF4A57216A11BA056
:1064F000F9F75EFF0720FFF759FA05004FF000009B
:1065000008D0CDE9004033461A463946284600F007
:1065100085FB2846BDE8FC812E2E2F4D6964646CF6
:106520006577617265732F54686972645F50617238
:1065300074792F4C7749502F7372632F636F726594
:106540002F706275662E6300696E76616C696420D7
:10655000706275665F7479706500000041737365E1
:106560007274696F6E2022257322206661696C65E2
:1065700064206174206C696E6520256420696E203A
:1065800025730A007CB51C46DDE90635C01C20F0E9
:1065900003004618AE4201D900207CBD0BB118445F
:1065A00000E000200223CDE900230B4601461A46F5
:1065B000204600F033FB20467CBD000070B50D4640
:1065C00008B1002D08D1BDE8704014A340F2593243
:1065D0001EA12CA0F9F7ECBE0446006820B1218969
:1065E0002A8911442181F7E72089618988420FD0E7
:1065F0000AA340F262322DA122A0F9F7D9FE206849
:1066000030B106A340F2633234A11EA0F9F7D0FEE8
:106610002089298908442081256070BD2E2E2F4DA8
:106620006964646C6577617265732F54686972641C
:106630005F50617274792F4C7749502F7372632FBA
:10664000636F72652F706275662E63002868202163
:106650003D204E554C4C2920262620287420213DD3
:10666000204E554C4C29202870726F6772616D6DF9
:1066700065722076696F6C61746573204150492999
:1066800000000000417373657274696F6E202225EB
:106690007322206661696C6564206174206C696E88
:1066A0006520256420696E2025730A00702D3E74D4
:1066B0006F745F6C656E203D3D20702D3E6C656E85
:1066C00020286F66206C6173742070627566206983
:1066D0006E20636861696E2900000000702D3E6EB7
:1066E000657874203D3D204E554C4C00002102E061
:1066F000491C006889B20028FAD10846704700009A
:1067000070B5154613890A461946FFF7C9FD0400FE
:106710000CD0294600F042F830B105A340F22452D3
:106720000FA114A0F9F744FE204670BD002070BDF3
:106730002E2E2F4D6964646C6577617265732F54DA
:10674000686972645F50617274792F4C7749502F79
:106750007372632F636F72652F706275662E6300AC
:10676000706275665F636F7079206661696C6564DD
:1067700000000000417373657274696F6E202225FA
:106780007322206661696C6564206174206C696E97
:106790006520256420696E2025730A002DE9F047E5
:1067A0004FF000070C4605003E466FF00F0904D07D
:1067B0001CB128892189884204D232A340F2C9320F
:1067C0003CA145E06FF0050A6889C11B6089801B08
:1067D000814201D3804600E08846606842468119C4
:1067E00068683844F9F7F3FE688947444644B8427C
:1067F00006D224A340F2D9323AA140A0F9F7D8FD3D
:106800006089B04206D21FA340F2DA3245A13BA014
:10681000F9F7CEFD6089B04201D824680026688966
:10682000B84202D12D68002765B1002C16D06089CE
:106830002189884212D1206800280FD011A340F28C
:10684000E93215E0002C1BD00EA34FF479723CA165
:106850002AA0F9F7ADFD4846BDE8F08775B1688913
:10686000298988420AD1286840B106A340F2EE3255
:1068700037A122A0F9F79CFD5046EDE7002CA3D1EB
:106880000020E9E72E2E2F4D6964646C65776172F4
:1068900065732F54686972645F50617274792F4C0C
:1068A0007749502F7372632F636F72652F70627513
:1068B000662E6300706275665F636F70793A20744C
:1068C0006172676574206E6F742062696720656EFF
:1068D0006F75676820746F20686F6C6420736F75C4
:1068E000726365006F66667365745F746F203C3D0C
:1068F00020705F746F2D3E6C656E00004173736590
:106900007274696F6E2022257322206661696C653E
:1069100064206174206C696E6520256420696E2096
:1069200025730A006F66667365745F66726F6D200B
:106930003C3D20705F66726F6D2D3E6C656E000091
:10694000705F746F20213D204E554C4C00000000BC
:10695000706275665F636F7079282920646F657354
:10696000206E6F7420616C6C6F77207061636B6553
:106970007420717565756573210000002DE9F0477D
:10698000002716468946B84620B1B9F1000F06D057
:1069900004462CE018A340F20A4223A103E016A308
:1069A00040F20B4228A131A0F9F702FD0020BDE81A
:1069B000F0872BB16089984202D8181A83B215E08B
:1069C0006089C01A85B2B54200D9354660682A464A
:1069D000C11809EB0700F9F7FAFD08EB05001FFAEB
:1069E00080F8781987B2701B86B2002324680EB134
:1069F000002CDED14046DAE72E2E2F4D6964646C00
:106A00006577617265732F54686972645F50617253
:106A100074792F4C7749502F7372632F636F7265AF
:106A20002F706275662E6300706275665F636F70AB
:106A3000795F7061727469616C3A20696E76616C1D
:106A40006964206275660000706275665F636F70CE
:106A5000795F7061727469616C3A20696E76616CFD
:106A600069642064617461707472000041737365BD
:106A70007274696F6E2022257322206661696C65CD
:106A800064206174206C696E6520256420696E2025
:106A900025730A0070B5040003D00025A07B48B11F
:106AA0000FE024A34FF437722EA131A0F9F780FC38
:106AB000002070BD1FA340F2F12237A12CA0F9F7EE
:106AC00077FCA07B401E10F0FF00A07323D1207B39
:106AD000617B266800F00F0089070CD5206930B96A
:106AE00014A340F2FF2232A121A0F9F761FC216931
:106AF000204688470BE002280FD0012810D0A0B113
:106B00000CA340F20F3233A119A0F9F751FC6D1C10
:106B1000EDB23400C2D1284670BD2146082001E004
:106B200021460720FEF78AFEF1E72046FEF792FB9A
:106B3000EDE700002E2E2F4D6964646C657761725D
:106B400065732F54686972645F50617274792F4C59
:106B50007749502F7372632F636F72652F70627560
:106B6000662E63007020213D204E554C4C000000E5
:106B7000417373657274696F6E20222573222066DB
:106B800061696C6564206174206C696E65202564A0
:106B900020696E2025730A00706275665F667265F3
:106BA000653A20702D3E726566203E203000000060
:106BB00070632D3E637573746F6D5F667265655F9C
:106BC00066756E6374696F6E20213D204E554C4C86
:106BD00000000000696E76616C6964207062756601
:106BE000207479706500000010B501460448FEF776
:106BF00073FE04480178012901D10021017010BD04
:106C0000E0C00008000000200122AFF3008000294E
:106C100002DA494200F0F0B8FFF7E2BA70B500249A
:106C2000DDE90456C0E900410281438105734673E2
:106C300001218173C47370BD2DE9F0410D4604003C
:106C400006D121A34FF4CC722BA131A0F9F7B0FBF0
:106C50002089A84235D9401B86B240F2AF170CE01C
:106C6000281A85B22089801B208124682CB916A39C
:106C70003A4631A126A0F9F79BFB6089A842EFD3E1
:106C8000207B000715D16089A84212D0607B800765
:106C90000FD4A088001B284481B22046FEF7ECFCEC
:106CA000040006D108A340F2BD1229A118A0F9F7EB
:106CB0007FFB65812581206808B1FFF7EBFE00208E
:106CC0002060BDE8F08100002E2E2F4D6964646CB9
:106CD0006577617265732F54686972645F50617281
:106CE00074792F4C7749502F7372632F636F7265DD
:106CF0002F706275662E6300706275665F726561E3
:106D00006C6C6F633A207020213D204E554C4C0036
:106D1000417373657274696F6E2022257322206639
:106D200061696C6564206174206C696E65202564FE
:106D300020696E2025730A00706275665F72656156
:106D40006C6C6F633A207120213D204E554C4C00F5
:106D50006D656D5F7472696D2072657475726E65B4
:106D6000642071203D3D204E554C4C0000280CD035
:106D7000817B491C11F0FF01817306D103A340F20E
:106D800042320EA112A0F9F713BB70472E2E2F4DE1
:106D90006964646C6577617265732F5468697264A5
:106DA0005F50617274792F4C7749502F7372632F43
:106DB000636F72652F706275662E63007062756610
:106DC00020726566206F766572666C6F77000000D2
:106DD000417373657274696F6E2022257322206679
:106DE00061696C6564206174206C696E652025643E
:106DF00020696E2025730A0010B520B1B1F5803FDF
:106E000006D3012010BD0FA340F24B2219A109E0C7
:106E100000290BD043898AB2934209D209A340F2D8
:106E2000552217A11EA0F9F7C3FAEAE7002010BD0A
:106E3000446821444160991A41810189891A01817C
:106E4000F4E700002E2E2F4D6964646C6577617243
:106E500065732F54686972645F50617274792F4C46
:106E60007749502F7372632F636F72652F7062754D
:106E7000662E63007020213D204E554C4C000000D2
:106E8000696E6372656D656E745F6D61676E69745E
:106E9000756465203C3D20702D3E6C656E000000E1
:106EA000417373657274696F6E20222573222066A8
:106EB00061696C6564206174206C696E652025646D
:106EC00020696E2025730A002DE9F041304D0446FB
:106ED0002868844206D22FA340F2DF1239A13FA0D6
:106EE000F9F766FA6868844206D32AA34FF4F07271
:106EF00044A13AA0F9F75CFA207930B125A340F219
:106F0000E11247A135A0F9F753FA20884FF4C86879
:106F1000404506D91FA34FF4F27248A12FA0F9F7FC
:106F200047FA208800F0A0F80646B44215D0307920
:106F300098B96868864210D0A868B04200D1AC60A9
:106F4000308820803088404507D02046FEF78CFBF3
:106F50000746308800F088F84780608800F084F8A1
:106F6000A04212D0017900290FD1A968A14200D115
:106F7000A860218801802188414506D0FEF774FB76
:106F80000546208800F070F84580BDE8F0810000DB
:106F9000480000202E2E2F4D6964646C6577617265
:106FA00065732F54686972645F50617274792F4CF5
:106FB0007749502F7372632F636F72652F6D656D04
:106FC0002E630000706C75675F686F6C65733A20A4
:106FD0006D656D203E3D2072616D000041737365EB
:106FE0007274696F6E2022257322206661696C6558
:106FF00064206174206C696E6520256420696E20B0
:1070000025730A00706C75675F686F6C65733A2052
:107010006D656D203C2072616D5F656E64000000DF
:10702000706C75675F686F6C65733A206D656D2D68
:107030003E75736564203D3D20300000706C7567BF
:107040005F686F6C65733A206D656D2D3E6E657877
:1070500074203C3D204D454D5F53495A455F414C9E
:1070600049474E45440000000149096808447047FB
:1070700048000020FBF7DAB870B515460E46044606
:10708000B0F1804F06D308A340F2291213A121A02A
:10709000F9F78EF9FFF7EEFF20442A463146BDE8A6
:1070A000704000F04BB800002E2E2F4D6964646CC8
:1070B0006577617265732F54686972645F5061729D
:1070C00074792F4C7749502F7372632F636F7265F9
:1070D0002F74696D656F7574732E630054696D65E7
:1070E0006F75742074696D6520746F6F206C6F6E9E
:1070F000672C206D6178206973204C5749505F558B
:10710000494E5433325F4D41582F34206D736563BF
:1071100073000000417373657274696F6E202225DD
:107120007322206661696C6564206174206C696EED
:107130006520256420696E2025730A0070B5044619
:1071400015460E460620FEF731FC78B10021C560D9
:10715000104A80E85200116831B14B68E51A4FF0CF
:1071600000439D4212D30160106070BDBDE87040C5
:1071700009A3BE2215A125A0F9F71AB95568651B08
:107180009D4202D30260086070BD11460A68002A61
:10719000F8D0F3E7CC0000202E2E2F4D6964646CEC
:1071A0006577617265732F54686972645F506172AC
:1071B00074792F4C7749502F7372632F636F726508
:1071C0002F74696D656F7574732E63007379735FC7
:1071D00074696D656F75743A2074696D656F757447
:1071E00020213D204E554C4C2C20706F6F6C204D53
:1071F000454D505F5359535F54494D454F555420A9
:10720000697320656D7074790000000041737365C7
:107210007274696F6E2022257322206661696C6525
:1072200064206174206C696E6520256420696E207D
:1072300025730A0070B5074D012400BF05EBC40299
:1072400055F834000449FFF717FF641C032CF5D3ED
:1072500070BD0000F4C10008E15100082DE9FF5F96
:107260008946040003D0207D01280AD010E004B034
:107270003AA3BDE8F05F40F23D2244A14AA0F9F7ED
:1072800097B836A34FF4107251A147A0F9F790F8C0
:10729000207D0A283ED0216D03910025DFF864810E
:1072A000D4F824B0D4F810A0D4F890602F4680B35E
:1072B0004D46E78A214608F1180002F069FA0121DB
:1072C00088F80010206F08B103F098FEE06E08B156
:1072D00003F094FE606F08B103F090FE55B1208B6F
:1072E000211D0091CDE9017023465A4618460399A5
:1072F00003F096FD204600F029FD002E2CD004B0AE
:107300005046B446BDE8F04F6FF00C015DF804EB59
:1073100060470AE03B4821461C3002F039FA04B0CD
:107320002046BDE8F05F00F011BDE08A0028C9D01A
:10733000D8F81000A0420AD1C068C8F8100008E0D0
:10734000C168A14202D1E168C16002E0084600289C
:10735000F6D10020E060B5E7BDE8FF9F2E2E2F4D4F
:107360006964646C6577617265732F5468697264CF
:107370005F50617274792F4C7749502F7372632F6D
:10738000636F72652F7463702E6300007463705FA7
:107390006162616E646F6E3A20696E76616C6964D9
:1073A0002070636200000000417373657274696F3E
:1073B0006E2022257322206661696C6564206174E9
:1073C000206C696E6520256420696E2025730A0093
:1073D000646F6E27742063616C6C207463705F61EE
:1073E000626F72742F7463705F6162616E646F6E3E
:1073F00020666F72206C697374656E2D70636273A2
:1074000000000000880000200121FFF727BF0000D6
:107410002DE9F04106460120FEF7C8FA424D04006E
:107420005BD1A86909E0418BC4680A0704D521F043
:107430000801418300F0BCF920460028F3D1002266
:107440001146EC68E86906E0036AE31A934201D347
:107450001A460146C0680028F6D111B10846FFF768
:10746000D3FF0120FEF7A2FA040036D1092001F073
:1074700075F90120FEF79AFA04002ED1082001F0D8
:107480006DF90120FEF792FA040026D17F2E01D972
:107490007F2001E030001BD0401EC1B200231A46FD
:1074A000EC68A8690EE0477D8F4206D309D1D0F879
:1074B00020C0A4EB0C0C9C4503D3016A0246631A5E
:1074C0003946C0680028EED112B11046FFF79CFF84
:1074D0000120FEF76BFA040023D09C21F9F7BCF8D9
:1074E0004FF486606675A4F86400410061852185CB
:1074F000FF21E172411061860621A4F84010E18766
:10750000C91F21860121A4F84810E9682162A978E1
:10751000A177A4F84A000548C4F884000448C4F8D8
:1075200094002046BDE8F08188000020EDA7000807
:1075300000DD6D0010B558B1017D012903D0418BEC
:1075400041F010014183BDE81040012100F042B834
:1075500004A34FF4F4720FA114A0F8F729FF6FF001
:107560000F0010BD2E2E2F4D6964646C657761721B
:1075700065732F54686972645F50617274792F4C1F
:107580007749502F7372632F636F72652F74637026
:107590002E6300007463705F636C6F73653A2069DB
:1075A0006E76616C6964207063620000417373657C
:1075B0007274696F6E2022257322206661696C6582
:1075C00064206174206C696E6520256420696E20DA
:1075D00025730A00FEB50D46040006D145A34FF4FD
:1075E000AF7250A157A0F8F7E3FE28005F4D4FF0AF
:1075F00000064FF001073ED0207D042801D0072867
:1076000039D1A06F18B9208DB0F5066F33D0A07EA8
:10761000C00606D437A34FF4B27255A149A0F8F7BB
:10762000C7FE228BE18A201D8DE8070023461846FD
:10763000626A216D03F0F4FB204602F043F8A8696A
:10764000A04209D1C068A86108E0C168A14202D186
:10765000E168C16002E008460028F6D14B48E660C8
:107660002F700068A04202D104F056FA38E020469C
:1076700000F06CFB34E0207D40B101281AD00228D4
:1076800030D02046BDE8FE4000F092B8E08A0028E5
:10769000EDD02869A04209D1C068286108E0C1681E
:1076A000A14202D1E168C16002E008460028F6D19B
:1076B000E660DCE7204601F0AFF82C4821461430A4
:1076C00002F066F8207D012806D1314BDF2231A17E
:1076D00003F14400F8F76CFE21460220FEF7AEF8F5
:1076E0000020FEBD21482146183002F051F82F70CD
:1076F000BDE700002E2E2F4D6964646C65776172C2
:1077000065732F54686972645F50617274792F4C8D
:107710007749502F7372632F636F72652F74637094
:107720002E6300007463705F636C6F73655F7368D2
:107730007574646F776E3A20696E76616C69642047
:1077400070636200417373657274696F6E202225E5
:107750007322206661696C6564206174206C696EB7
:107760006520256420696E2025730A0088000020AA
:107770007063622D3E666C61677320262054465FFD
:107780005258434C4F53454400000000C8000020AD
:10779000707D00087463705F667265655F6C697305
:1077A00074656E3A20214C495354454E0000000048
:1077B00070B5050006D116A34FF4CE7220A123A008
:1077C000F8F7F6FD287D0526032804D0042802D00A
:1077D000072816D106E0284603F090FC040006D1E5
:1077E0002E7509E0284603F089FC040002D0601CD5
:1077F00009D004E009202875284601F069FA2046DE
:1078000070BD002070BD688B40F008006883F8E709
:107810002E2E2F4D6964646C6577617265732F54E9
:10782000686972645F50617274792F4C7749502F88
:107830007372632F636F72652F7463702E63000021
:1078400070636220213D204E554C4C00417373659E
:107850007274696F6E2022257322206661696C65DF
:1078600064206174206C696E6520256420696E2037
:1078700025730A002DE9F047DDF820809A469146ED
:107880000D46070005D12DA3A32239A140A0F8F78A
:107890008FFD002D05D129A3A42247A13CA0F8F714
:1078A00087FD5FEAC87001D0042600E000260320AF
:1078B000FEF77CF804001CD084F80A804FF0000822
:1078C000C4E900852889B04205D21CA3B02243A197
:1078D0002FA0F8F76DFD28891421801B20812846F0
:1078E000FEF77AFC48B1204603F07AFB0020BDE8A1
:1078F000F0872846FFF7CEF8F8E760684068E06058
:10790000F88AFDF78DFCE1680880388BFDF788FC6C
:10791000E16848805046FDF781FCE1684860B008A6
:10792000000300F5A04040EA0900FDF779FCE1689A
:107930008881E1682046A1F81280D8E72E2E2F4DCD
:107940006964646C6577617265732F5468697264E9
:107950005F50617274792F4C7749502F7372632F87
:10796000636F72652F7463705F6F75742E630000B0
:107970007463705F6372656174655F7365676D657D
:107980006E743A20696E76616C696420706362007F
:10799000417373657274696F6E20222573222066AD
:1079A00061696C6564206174206C696E6520256472
:1079B00020696E2025730A007463705F63726561CD
:1079C00074655F7365676D656E743A20696E766184
:1079D0006C6964207062756600000000702D3E7452
:1079E0006F745F6C656E203E3D206F70746C656EC9
:1079F0000000000070B50C460546002A06D10BA316
:107A000040F6C50215A11FA0F8F7D2FC5CB1A18C0D
:107A100049B1282902D928398CB200E00024A542B6
:107A200000D22C462546284670BD00002E2E2F4D34
:107A30006964646C6577617265732F5468697264F8
:107A40005F50617274792F4C7749502F7372632F96
:107A5000636F72652F7463702E6300007463705FD0
:107A60006566665F73656E645F6D73735F6E657484
:107A700069663A20696E76616C6964206473745F2C
:107A800069700000417373657274696F6E202225FE
:107A90007322206661696C6564206174206C696E74
:107AA0006520256420696E2025730A002DE9F843BE
:107AB000044600250E46880706D13FA340F2114236
:107AC0004A494BA0F8F774FC002C06D13AA340F2C7
:107AD000134251A146A0F8F76BFCB00700D5012571
:107AE000E80700D00420804601464FF4207236207B
:107AF000FEF7D6FB07004FF0FF3929D079894145C1
:107B000006D22DA340F239424BA139A0F8F750FC20
:107B10000095324639462046E36DFFF7ABFE05007F
:107B200016D0287B800706D023A340F2424251A101
:107B30002FA0F8F73DFC2889002806D01EA340F2AC
:107B4000434252A12AA0F8F733FCE06E38B109E0B5
:107B5000608B40F0800060834846BDE8F883E566AE
:107B600004E0084601680029FBD105600020A4F864
:107B70006800B00702D0E06D401CE065F00703D05C
:107B8000608B40F0200060836868FEF7AFFDB4F8BA
:107B9000661008440004000CA4F866000AD0206FA8
:107BA00040B9E06E30B904A340F2654242A110A092
:107BB000F8F7FEFB0020D0E72E2E2F4D6964646C91
:107BC0006577617265732F54686972645F50617282
:107BD00074792F4C7749502F7372632F636F7265DE
:107BE0002F7463705F6F75742E63000094C2000879
:107BF000417373657274696F6E202225732220664B
:107C000061696C6564206174206C696E652025640F
:107C100020696E2025730A007463705F656E71754C
:107C20006575655F666C6167733A20696E76616C35
:107C300069642070636200007463705F656E7175C3
:107C40006575655F666C6167733A20636865636B31
:107C5000207468617420666972737420706275663E
:107C60002063616E20686F6C64206F70746C656E49
:107C7000000000007365672D3E74637068647220B5
:107C80006E6F7420616C69676E6564007463705F09
:107C9000656E71756575655F666C6167733A2069BD
:107CA0006E76616C6964207365676D656E74206CB7
:107CB000656E6774680000007463705F656E71754F
:107CC0006575655F666C6167733A20696E76616C95
:107CD0006964207175657565206C656E67746800F0
:107CE00070B5194DA878401CA870AC6928E0A17F38
:107CF000A878814223D0A077608BC10709D040F0DB
:107D000002006083204600F0E3FF608B20F0030058
:107D1000608380B2010705D520F00800608320460B
:107D2000FFF746FDE668A06F38B1002028702046B6
:107D300002F058F828780028D7D1344600E0E468EB
:107D4000002CD4D170BD00008800002010B504467E
:107D5000007D012805D106A3D42211A115A0F8F7B2
:107D600027FB2146BDE810400120FDF767BD00005C
:107D70002E2E2F4D6964646C6577617265732F5484
:107D8000686972645F50617274792F4C7749502F23
:107D90007372632F636F72652F7463702E630000BC
:107DA0007463705F667265653A204C495354454E62
:107DB00000000000417373657274696F6E202225A4
:107DC0007322206661696C6564206174206C696E41
:107DD0006520256420696E2025730A002DE9F0478F
:107DE00099460C460646224F2AE02546D5E9004032
:107DF000FEF77CFCB6F866108046414506D21DA30E
:107E000040F2574228A132A0F8F7D2FA36F8661F9E
:107E1000A1EB080030802889398908443881284638
:107E200003F0DEF836F86609002809D054EA0900A4
:107E300006D110A340F261422FA125A0F8F7B8FAAD
:107E400094B1E0684068FDF7E9F90546E06880898B
:107E5000FDF7E6F9800700D0012021892844084475
:107E6000B969401A0028C0DD2046BDE8F08700004F
:107E7000A80000202E2E2F4D6964646C6577617216
:107E800065732F54686972645F50617274792F4C06
:107E90007749502F7372632F636F72652F7463700D
:107EA0005F696E2E630000007063622D3E736E6426
:107EB0005F71756575656C656E203E3D20706275FD
:107EC000665F636C656E286E6578742D3E70290060
:107ED000417373657274696F6E2022257322206668
:107EE00061696C6564206174206C696E652025642D
:107EF00020696E2025730A007463705F7265636584
:107F00006976653A2076616C69642071756575657E
:107F1000206C656E6774680010B50446406F0028D9
:107F200003D003F06BF80020606710BD0849C888D3
:107F3000421CCA800A6912B18B88984203D2C96870
:107F40001431085C7047C01AC0B2105C7047000062
:107F5000A800002010B5F8F779F90349C0F30D0027
:107F600000F54040888010BD880000202DE9FE4FBC
:107F7000040005D1DEA38322EAA1F0A0F8F718FAE5
:107F8000F84D6068E860608914287DD3F64E31684A
:107F90007069FCF7E9F8002876D1307DB046C0F36F
:107FA00003100E2870D0E8688089FDF739F9000BBE
:107FB00081001429E9D320898842E6D3A1F1140075
:107FC00080B268804FF0000AC5F810A062898A422A
:107FD00004D3A8802046FEF70FFF32E0206828B9BE
:107FE000C3A3C222E1A1D5A0F8F7E2F914212046EB
:107FF000FEF702FF6189A9806888401A86B2204690
:10800000FEF7FAFE20684189B142BED3416829617A
:108010003146FEF7F1FE2089801B2081608928B15E
:10802000B3A3DF22D5A1C5A0F8F7C2F92168208942
:108030000989884205D0AEA3E022D3A1BFA0F8F7FA
:10804000B7F9E8680088FDF7EBF80146E8680180B9
:108050004088FDF7E5F80146E86841804068FDF793
:10806000DDF80146E868416069618068FDF7D6F88F
:108070000146E8688160A961C089FDF7D1F8014631
:10808000E868C181808900E08CE0FDF7C9F800F064
:108090003F01297020896881890704D0411C89B279
:1080A000698188427ED8DFF800930027D9F8006004
:1080B00083E0307D28B98EA3FB22BCA19FA0F8F7F6
:1080C00077F9307D0A2805D189A3FC22C1A19BA0A4
:1080D000F8F76EF9307D012805D185A3FD22C8A1EE
:1080E00096A0F8F765F9307A38B1D8F8041091F80D
:1080F0003010491CC9B288425DD1E868318B0288D2
:10810000914258D1F18A4088814254D17168D8F89F
:10811000102091424FD13168D8F8140081424AD1E1
:10812000F068B04206D172A340F20D12BEA183A046
:10813000F8F73EF937B1F068F860D9F80010F1604F
:10814000C9F80060F068B04206D169A340F2151288
:10815000C0A17AA0F8F72CF996B3DFF8248357462C
:10816000C8F800A02189A8F80810C8F80440E968F8
:10817000C8F80C10C5F81CA085F801A0A5F808A047
:108180002878000703D5607B40F001006073B06F72
:10819000002878D0304601F025FE0D3007D0B06FB2
:1081A000002800E0F5E16ED0688900286BD0708D62
:1081B000002864D0CCE13746F668002E7FF479AF12
:1081C000B04840F21F194646076827E0387D0A2864
:1081D00005D047A34A46ACA158A0F8F7E9F8387A89
:1081E00030B1716891F83010491CC9B2884214D17D
:1081F000E8683A8B01888A420FD1F98A4088814227
:108200000BD178683169884207D138687169884232
:1082100003D1384603F0F0FBBBE1FF68002FD5D156
:10822000A54B0021EF681868D6F804900246D6F8EE
:10823000148016E0067A3EB199F830C00CF1010CBA
:108240000CF0FF0C66450AD1C68AB7F802C0664535
:1082500005D10668464507D0002804D036B101464E
:10826000C0680028E6D17FE100283FD019B1C56879
:10827000CD60C260186000F007FB8AE103E0304681
:1082800002F0C6FE64E130462E6201F049FB0D307B
:1082900011D068782C4600070ED5D6F890201AB178
:1082A0006FF00D013069904731463F4801F070FA98
:1082B0003046FFF74BFD4BE1228942B1D6F88030C2
:1082C00023B13146306998470D300CD027813046B4
:1082D00000F074F938B9E06930B1B06F28B104A387
:1082E0004FF4F372EAE033E10EE1ECE03CE1000030
:1082F0002E2E2F4D6964646C6577617265732F54FF
:10830000686972645F50617274792F4C7749502F9D
:108310007372632F636F72652F7463705F696E2E63
:10832000630000007463705F696E7075743A206951
:108330006E76616C69642070627566004173736566
:108340007274696F6E2022257322206661696C65E4
:1083500064206174206C696E6520256420696E203C
:1083600025730A00A8000020404D0020702D3E6EAD
:1083700065787420213D204E554C4C00702D3E6C8C
:10838000656E203D3D203000702D3E746F745F6C33
:10839000656E203D3D20702D3E6E6578742D3E74D7
:1083A0006F745F6C656E0000A00000207463705FE6
:1083B000696E7075743A20616374697665207063C4
:1083C000622D3E737461746520213D20434C4F53F0
:1083D000454400007463705F696E7075743A206183
:1083E0006374697665207063622D3E737461746591
:1083F00020213D2054494D452D574149540000004E
:108400007463705F696E7075743A20616374697625
:1084100065207063622D3E737461746520213D2078
:108420004C495354454E00007463705F696E70751B
:10843000743A207063622D3E6E65787420213D2071
:1084400070636220286265666F726520636163688D
:10845000652900007463705F696E7075743A2070EE
:1084600063622D3E6E65787420213D20706362202A
:108470002861667465722063616368652900000085
:108480006C820020A40000207463705F696E7075B8
:10849000743A2054494D452D574149542070636228
:1084A0002D3E7374617465203D3D2054494D452D2A
:1084B00057414954000000009C00002037A1AFF252
:1084C0008410F7F775FFB07EC00606D5E069FEF7A9
:1084D000E1FA3046FEF798FF3AE0D6F884C0BCF1E6
:1084E000000F05D0002330693146E269E04705E01E
:1084F000002331461846E26902F078F910F10D0FB9
:1085000026D008B1E069B0676078800618D5B06FF2
:1085100020B1417B41F02001417311E0308DB0F575
:10852000066F01D0401C3085D6F884C0BCF1000F26
:1085300006D000231A4631463069E0470D3007D097
:108540003046276200F03AF810B9304600F0C0FB20
:108550002F62EF61D8F804004446002802D0FEF7ED
:1085600099FA6760BDE8FE8FB889FCF759FE4007AD
:108570000FD4E868104A104B018840880092CDE97A
:108580000101698968691B1D42180020A96902F070
:1085900047FC2046BDE8FE4FFEF77CBA7063622DB3
:1085A0003E726566757365645F64617461203D3D0C
:1085B000204E554C4C000000504D002010B50400DA
:1085C00006D110A340F25A221BA125A0F7F7F0FE16
:1085D0002D484078C00612D5A07EC00606D4D4F837
:1085E00090201AB16FF00E0120699047214627486C
:1085F00001F0CEF82046FFF7A9FB012010BD0020B6
:1086000010BD00002E2E2F4D6964646C6577617279
:1086100065732F54686972645F50617274792F4C6E
:108620007749502F7372632F636F72652F74637075
:108630005F696E2E630000007463705F696E707511
:10864000745F64656C617965645F636C6F73653AD0
:1086500020696E76616C69642070636200000000BE
:10866000417373657274696F6E20222573222066D0
:1086700061696C6564206174206C696E6520256495
:1086800020696E2025730A00A8000020A0000020A9
:1086900070B504004FF0000606D112A340F6240284
:1086A0001DA124A0F7F784FE206D401EFCF7B6FD47
:1086B000034600223146204600F07AFC05000DD02A
:1086C000014633460022204600F0D0FD2246231DFD
:1086D0002946BDE87040104600F058BD4FF0FF300D
:1086E00070BD00002E2E2F4D6964646C6577617239
:1086F00065732F54686972645F50617274792F4C8E
:108700007749502F7372632F636F72652F74637094
:108710005F6F75742E6300007463705F6B656570C6
:10872000616C6976653A20696E76616C6964207067
:1087300063620000417373657274696F6E20222555
:108740007322206661696C6564206174206C696EB7
:108750006520256420696E2025730A0070B50446E3
:10876000082808D0092C06D010A340F2DD621BA116
:108770001EA0F7F71DFE274B002108469A69DB680B
:1087800009E0157DA54205D1156A5D1B8D4201D317
:1087900029461046D268002AF3D1002804D0BDE84B
:1087A00070400021FEF75ABD70BD00002E2E2F4DE7
:1087B0006964646C6577617265732F54686972646B
:1087C0005F50617274792F4C7749502F7372632F09
:1087D000636F72652F7463702E630000696E76613B
:1087E0006C69642073746174650000004173736583
:1087F0007274696F6E2022257322206661696C6530
:1088000064206174206C696E6520256420696E2087
:1088100025730A008800002070B5050007D10F4BB2
:1088200040F211120EA103F14400F7F7C1FD287DBB
:10883000012807D0094B4FF489720CA103F14400C1
:10884000F7F7B6FD0F4E0124294656F824000068BC
:1088500002F0A4F8641C042CF6D370BD707D0008EF
:1088600070636220213D204E554C4C007063622D98
:108870003E7374617465203D3D204C495354454E10
:1088800000000000E4C10008FEB5424E0546307805
:1088900040071BD4002D06D13FA340F281224BA1FB
:1088A00052A0F7F785FD3078C10610D5F068594A17
:1088B000584B018840880092CDE9010171897069A7
:1088C0001B1D42182846B16902F0AAFAFEBD8007B6
:1088D000FCD5687DFEF79CFD04004AD04D48103859
:1088E0004169216000696060E88AE082F068008880
:1088F0002083032020757069401C6062E06220467E
:1089000000F014F9A06520656064E0657069401EA0
:1089100060652869E5672061687A00F00C00607284
:10892000287A20723C480168E160046003F04AF84C
:108930003A4901200870204600F046FEF068C089E0
:10894000A4F86000A4F86200201DFCF735F8014689
:10895000608E221DFFF74EF8608612212046FFF739
:10896000A5F888B103B02046BDE8F0400021FEF72D
:1089700075BCAB69002BA9D0286903B04FF0FF325A
:10898000BDE8F040002118472046BDE8FE4000F059
:108990009FB90000A80000202E2E2F4D6964646C42
:1089A0006577617265732F54686972645F50617294
:1089B00074792F4C7749502F7372632F636F7265F0
:1089C0002F7463705F696E2E630000007463705FC4
:1089D0006C697374656E5F696E7075743A20696E48
:1089E00076616C6964207063620000004173736596
:1089F0007274696F6E2022257322206661696C652E
:108A000064206174206C696E6520256420696E2085
:108A100025730A00504D0020A0000020880000208F
:108A200070B50D4604001DD0206800281AD00E4EE7
:108A30002046B16900F01AF82046316900F016F8B6
:108A4000002D0FD0286800280CD006F11400026811
:108A500006E010682168884201D128681060D26859
:108A6000002AF6D170BD00008800002070B5050016
:108A70000C4612D10AA34FF4106215A121A0F7F7FA
:108A800097FC0AE020682968884205D12046E668FC
:108A9000FEF7BAFC344600E0E468002CF2D170BD69
:108AA0002E2E2F4D6964646C6577617265732F5447
:108AB000686972645F50617274792F4C7749502FE6
:108AC0007372632F636F72652F7463702E6300007F
:108AD0007463705F6E657469665F69705F6164641A
:108AE000725F6368616E6765645F7063626C69730F
:108AF000743A20696E76616C6964206F6C645F61A2
:108B000064647200417373657274696F6E2022250C
:108B10007322206661696C6564206174206C696EE3
:108B20006520256420696E2025730A0010B5002891
:108B300006D106A340F6AF0210A117A0F7F738FC44
:108B40001F49D1E902021044886010BD2E2E2F4D1E
:108B50006964646C6577617265732F5468697264C7
:108B60005F50617274792F4C7749502F7372632F65
:108B7000636F72652F7463702E6300007463705F9F
:108B80006E6578745F6973733A20696E76616C699B
:108B90006420706362000000417373657274696FD2
:108BA0006E2022257322206661696C6564206174E1
:108BB000206C696E6520256420696E2025730A008B
:108BC0008800002070B50C46050006D11EA340F2B7
:108BD0001F422AA133A0F7F7EBFBE8688089FCF776
:108BE0001FFB3A4EC00715D0204602F007FA0024BA
:108BF00027E08089FCF714FBC00707D00120FCF7B1
:108C00000FFB0146E8688289114381812046246870
:108C100002F0E6F9ACB1E0682289736941680A4460
:108C200029891944891AE4D52989CA18E16849684B
:108C3000521A002A05DDC81A81B229816868FDF739
:108C4000FBFF2C6070BD00002E2E2F4D6964646CFC
:108C50006577617265732F54686972645F506172E1
:108C600074792F4C7749502F7372632F636F72653D
:108C70002F7463705F696E2E630000007463705F11
:108C80006F6F735F696E736572745F7365676D652F
:108C90006E743A20696E76616C69642063736567EF
:108CA00000000000417373657274696F6E202225A5
:108CB0007322206661696C6564206174206C696E42
:108CC0006520256420696E2025730A00A800002015
:108CD0002DE9F05F040006D187A340F2E14293A1A1
:108CE00098A0F7F765FB207D012806D182A340F20A
:108CF000E3429EA193A0F7F75BFBA6480068A04261
:108D000002D10020BDE8F09FB4F86010B4F848002C
:108D1000814200D20846E56E81466DB12146221D92
:108D2000084602F075F85FEA000A6FF003012ED0E2
:108D300054B1206840B10CE0A07E80076FD520467A
:108D4000BDE8F05F02F064B91AF104001FD00068BA
:108D50002060E8684068FCF761FA616C401A298974
:108D6000421800204A4514D9B4F860204A45E3D19E
:108D7000216F0029E0D194F899100029DCD184F802
:108D80009800012184F8991084F89A00D4E70846E5
:108D9000B8E784F89900266F83460EB998E0064636
:108DA00030680028FBD192E0E8688089FCF738FA47
:108DB000400706D550A340F2365277A161A0F7F7DD
:108DC000F7FA206FA8B1618B11F0440F11D1E06E5A
:108DD00028B102686AB90089628E904209D2B4F85B
:108DE000640030B1B4F86600092802D211F0A00F77
:108DF00079D0207D022807D01020FCF711FA014617
:108E0000E86882891143818152462146284600F054
:108E100099FA28B1618B41F08001618372E766E0C5
:108E20002868E066207D022803D0608B20F00300D4
:108E30006083E8684068FCF7F1F90746E8688089D4
:108E4000FCF7EEF9800700D0012029893844084456
:108E5000216D091A00D52065E8688089FCF7E0F9E2
:108E6000800700D001202989C8422CD0C5F800B065
:108E7000206F68B1E8684068FCF7D0F90746F068F1
:108E80004068FCF7CBF9381A1AD504F1700003E0FA
:108E9000256716E0D8F800008046006850B1C06829
:108EA0004068FCF7BBF90746E8684068FCF7B6F98C
:108EB000381AEFD4D8F800002860C8F8005005E050
:108EC00035602E4602E0284602F08AF8E56E55B17C
:108ED000E8684068FCF7A2F9616C401A29890144EE
:108EE00049457FF661AFE06E08B9A4F868B0608BC1
:108EF00020F08000608304E72E2E2F4D6964646C9F
:108F00006577617265732F54686972645F5061722E
:108F100074792F4C7749502F7372632F636F72658A
:108F20002F7463705F6F75742E6300007463705FDD
:108F30006F75747075743A20696E76616C6964201F
:108F400070636200417373657274696F6E202225CD
:108F50007322206661696C6564206174206C696E9F
:108F60006520256420696E2025730A00646F6E27D2
:108F7000742063616C6C207463705F6F75747075BE
:108F80007420666F72206C697374656E2D706362F5
:108F900073000000C8000020525354206E6F7420EC
:108FA000657870656374656420686572652100008A
:108FB0002DE9FF411D4616460F46040006D10EA3BB
:108FC00040F2427219A123A0F7F7F2F9E08A638D0B
:108FD0001022218B8DE80F002B4632463946606AFD
:108FE00000F04CF8002803D0628D616A1144E16200
:108FF00004B0BDE8F08100002E2E2F4D6964646C32
:109000006577617265732F54686972645F5061722D
:1090100074792F4C7749502F7372632F636F726589
:109020002F7463705F6F75742E6300007463705FDC
:109030006F75747075745F616C6C6F635F68656188
:109040006465723A20696E76616C6964207063624F
:1090500000000000417373657274696F6E202225F1
:109060007322206661696C6564206174206C696E8E
:109070006520256420696E2025730A002DE9F05FC4
:10908000834688180E46DDE90B98143081B21F46DE
:109090004FF420722220DDF828A0FDF701F9050029
:1090A0002AD0698906F11400814206D214A340F245
:1090B000237220A12BA0F7F77BF950466C68FCF7D0
:1090C000AFF820804846FCF7ABF8608067605846F0
:1090D000FCF7A4F8A060B008000300F5A04080B23F
:1090E00040EA0800FCF79CF8A0810D98FCF798F87E
:1090F000E0810020208260822846BDE8F09F0000C9
:109100002E2E2F4D6964646C6577617265732F54E0
:10911000686972645F50617274792F4C7749502F7F
:109120007372632F636F72652F7463705F6F7574F2
:109130002E630000636865636B2074686174206649
:109140006972737420706275662063616E20686F47
:109150006C6420737472756374207463705F6864E8
:1091600072000000417373657274696F6E2022256E
:109170007322206661696C6564206174206C696E7D
:109180006520256420696E2025730A00FEB51E4601
:1091900017460D00044606D112A340F287721EA1A5
:1091A00028A0F7F705F932463946204601F030FE8F
:1091B00018B12CB1E37AA17A04E06FF003040BE05C
:1091C000FF23002100910622CDE9012032463946D5
:1091D0002846FBF7E1F904462846FDF75BFC2046EC
:1091E000FEBD00002E2E2F4D6964646C65776172A0
:1091F00065732F54686972645F50617274792F4C83
:109200007749502F7372632F636F72652F74637089
:109210005F6F75742E6300007463705F6F75747098
:1092200075745F636F6E74726F6C5F7365676D6585
:109230006E743A20696E76616C696420706275663E
:1092400000000000417373657274696F6E202225FF
:109250007322206661696C6564206174206C696E9C
:109260006520256420696E2025730A0070B51546B7
:109270000C0006D10DA340F2567219A122A0F7F7F7
:1092800097F86068EA0700F1140100D00422104446
:109290001430884208D0BDE8704004A340F27572D3
:1092A00023A119A0F7F784B870BD00002E2E2F4D12
:1092B0006964646C6577617265732F546869726460
:1092C0005F50617274792F4C7749502F7372632FFE
:1092D000636F72652F7463705F6F75742E63000027
:1092E0007463705F6F75747075745F66696C6C5FC2
:1092F0006F7074696F6E733A20696E76616C696421
:109300002070627566000000417373657274696F46
:109310006E2022257322206661696C656420617469
:10932000206C696E6520256420696E2025730A0013
:109330006F7074696F6E73206E6F742066696C6CE9
:10934000656400002DE9FE4317460C46050006D172
:109350003DA34FF4B76249A150A0F7F729F8002CBC
:1093600006D139A340F2B95256A14CA0F7F720F824
:10937000002F06D134A340F2BA525AA147A0F7F702
:1093800017F8284600F0CCF810B10020BDE8FE83A5
:10939000606AFBF743FFE9688860608DFBF740FF78
:1093A000E968C881618D606A0844E062EE68A87A65
:1093B0001436C0070AD0221D39464FF40670FEF756
:1093C00019FB40F00170FBF729FF01C6B4F930002A
:1093D0004FF00008002801DAA4F83080606B38B93B
:1093E000494800686063E8684068FBF717FFA063BE
:1093F0006968A8898A88801A4A89121A4A81696824
:109400000A89101A08816968E8684860E968A1F863
:109410001080A87AE968C00700D0042014300844FE
:10942000B04206D008A340F21C6238A11BA0F6F798
:10943000BFFFA07A06218DE88300E37A221D214632
:109440006868FBF7A9F8A1E72E2E2F4D6964646CBC
:109450006577617265732F54686972645F506172D9
:1094600074792F4C7749502F7372632F636F726535
:109470002F7463705F6F75742E6300007463705F88
:109480006F75747075745F7365676D656E743A207F
:10949000696E76616C6964207365670041737365FA
:1094A0007274696F6E2022257322206661696C6573
:1094B00064206174206C696E6520256420696E20CB
:1094C00025730A007463705F6F75747075745F73D1
:1094D00065676D656E743A20696E76616C696420AB
:1094E000706362007463705F6F75747075745F731E
:1094F00065676D656E743A20696E76616C6964208B
:109500006E65746966000000940000206F707469D5
:109510006F6E73206E6F742066696C6C65640000FA
:1095200010B5040006D107A340F29A5212A11CA064
:10953000F6F73EFF6068807B012801D0012010BD56
:10954000002010BD2E2E2F4D6964646C657761720A
:1095500065732F54686972645F50617274792F4C1F
:109560007749502F7372632F636F72652F74637026
:109570005F6F75742E6300007463705F6F75747035
:1095800075745F7365676D656E745F627573793A44
:1095900020696E76616C6964207365670000000065
:1095A000417373657274696F6E2022257322206681
:1095B00061696C6564206174206C696E6520256446
:1095C00020696E2025730A002DE9F041060006D1BE
:1095D0001DA340F27D7229A12FA0F6F7E9FE384CB9
:1095E0006088002818D00020E0804FF406750FE056
:1095F000FEF79CFC00280FD0012809D002280DD0CE
:10960000FEF794FC022807D3E1880844801EE0801E
:10961000E08861888842EBD3BDE8F081FEF786FCE4
:109620000428F9D1E0886188801C8842F4D8FEF7CC
:109630007DFC0702FEF77AFC3843A84200D800B947
:1096400028467086E4E700002E2E2F4D6964646C76
:109650006577617265732F54686972645F506172D7
:1096600074792F4C7749502F7372632F636F726533
:109670002F7463705F696E2E630000007463705F07
:1096800070617273656F70743A20696E76616C698F
:109690006420706362000000417373657274696FC7
:1096A0006E2022257322206661696C6564206174D6
:1096B000206C696E6520256420696E2025730A0080
:1096C000A800002070B504001FD0207D00281BD00A
:1096D0000A2819D0012817D0A06F002510B1FDF776
:1096E000D9F9A567606F10B12046FEF715FC4FF061
:1096F000FF302086E06E01F081FC206F01F07EFCDF
:10970000E5662567A4F8685070BDBDE8704003A306
:1097100040F651020DA114A0F6F74ABE2E2E2F4D91
:109720006964646C6577617265732F5468697264EB
:109730005F50617274792F4C7749502F7372632F89
:10974000636F72652F7463702E6300007463705FC3
:109750007063625F70757267653A20696E76616CDE
:109760006964207063620000417373657274696F8D
:109770006E2022257322206661696C656420617405
:10978000206C696E6520256420696E2025730A00AF
:1097900070B50C00054606D129A340F6830234A11A
:1097A0003AA0F6F705FE002D06D125A340F6840267
:1097B00040A136A0F6F7FCFD2868A04209D1C06898
:1097C000286008E0C168A14202D1E168C16002E0FE
:1097D00008460028F6D100252046E560FFF772FF15
:1097E000207D0A280DD0012826D0608BC10708D023
:1097F00040F0020060832046FFF76AFA207D0128CE
:109800001AD0E06E30B10EA340F6930231A11FA032
:10981000F6F7CEFD206F30B109A340F6940233A1D4
:109820001AA0F6F7C5FD606F30B105A340F69602A9
:1098300035A116A0F6F7BCFD2575E58270BD0000C8
:109840002E2E2F4D6964646C6577617265732F5499
:10985000686972645F50617274792F4C7749502F38
:109860007372632F636F72652F7463702E630000D1
:109870007463705F7063625F72656D6F76653A20C6
:10988000696E76616C696420706362004173736510
:109890007274696F6E2022257322206661696C657F
:1098A00064206174206C696E6520256420696E20D7
:1098B00025730A007463705F7063625F72656D6F19
:1098C00076653A20696E76616C6964207063626CBB
:1098D00069737400756E73656E74207365676D656A
:1098E0006E7473206C65616B696E6700756E616381
:1098F0006B6564207365676D656E7473206C65615C
:109900006B696E67000000006F6F7365712073658F
:10991000676D656E7473206C65616B696E670000BE
:109920002DE9FE4F040006D1DDA34FF44772E9A1F3
:10993000EFA0F6F73DFDF84D287841072CD5217DA5
:10994000022905D0626A6869824206D189B117E0AE
:10995000206DA969884213D041E2811AFCD4218D7F
:109960001144401A0028F7DC608B40F0020060834D
:1099700035E2CBA34FF44E72E8A1DDA0F6F718FD57
:10998000687840F008006870608B20F00100608308
:109990006FF00D00BDE8FE8F800704D5207D022802
:1099A00001D00328E0D1A07EC00602D4E3480068BD
:1099B00020624FF0000884F89B8084F89A8020464B
:1099C000FFF702FEDE4B227D03F110000421DFF8D9
:1099D00074A3DD4FDD4E921E14334FF001094FF09A
:1099E0000A0B082AB8D2DFE802F00487F2F6EFF299
:1099F000EEED2A78D606AFD5920767D5626CAE69D0
:109A0000521CB24262D16869421C62626664E262C0
:109A1000EA68401ED289A4F86020A4F8622060653C
:109A20002175201DFAF7C8FF0146608E221DFDF743
:109A3000E1FF41F21C116086B1EB400F01D2420000
:109A400000E00A46B2EB800F01D9810003E0B1EBE0
:109A5000400F00D24100A4F84810B4F8660030B9B5
:109A60008FA34FF45B72BAA1A1A0F6F7A1FCB4F8E2
:109A70006600401EA4F86600256FBDB12868206707
:109A8000284601F0ADFA206FE0B1A4F8308084F8E8
:109A9000428000BFD4F88830002B3FF465AF00222D
:109AA0002146206998470D304DD05DE7E56E35B908
:109AB0007BA34FF45D72ACA18DA0F6F779FC28680A
:109AC000E066DDE74FF0FF302086E3E7E9680A88CB
:109AD00049888DE807006989686942182046A969A4
:109AE00001F09EF994F84200062804D2A4F83080D0
:109AF000204601F069F872E12A78D60657D5626CE3
:109B0000AE69B21A012A45D4226DB21A002A41DC8C
:109B10002175E06FA0B1806948B961A34FF46A7202
:109B200096A173A0F6F744FCE06F806940B1E16F45
:109B3000206900228B692146984738B10D3002D048
:109B40002046FDF761FC6FF00C0023E7204600F093
:109B5000CBF9288908B1401E2881618E41F21C1082
:109B6000B0EB410F01D24A0000E00246B2EB810F98
:109B700001D9880003E0B0EB410F00D24800A4F8FF
:109B800048006878800611D5608B40F00200608341
:109B9000072057E0E9680A8849888DE80700698945
:109BA000686942183146204601F03AF917E19007FA
:109BB00007D5606A6969401E884202D1204600F0DC
:109BC00019FF0CE1FBE057E03EE004E0FFE7204630
:109BD00000F08AF9D5E7204600F086F9687880061B
:109BE00028784FEAC06024D5002805DA206DA969DD
:109BF000884201D1E06E28B1608B40F002006083A2
:109C000008201FE0608B40F0020060832046FFF7D1
:109C100059FD3068A04209D1C0683060C5E0C16814
:109C2000A14202D1E168C160BFE008460028F6D138
:109C3000BBE0002833DA206DA96988422FD1E06E9D
:109C400068BB06202075CAE0204600F04DF9687810
:109C5000800624D5608B40F0020060832046FFF729
:109C600031FD3068A042D7D003E0C168A142D9D00D
:109C700008460028F9D198E0204600F035F9287808
:109C8000C0060CD5206DA969884208D1E06E30B9B4
:109C90002046FFF717FD3068A042BDD083E09EE06C
:109CA0002E2E2F4D6964646C6577617265732F5435
:109CB000686972645F50617274792F4C7749502FD4
:109CC0007372632F636F72652F7463705F696E2E9A
:109CD000630000007463705F70726F636573733A42
:109CE00020696E76616C6964207063620000000018
:109CF000417373657274696F6E202225732220662A
:109D000061696C6564206174206C696E65202564EE
:109D100020696E2025730A00A80000207463705F1C
:109D2000696E7075743A207063622D3E737461744D
:109D30006520213D20434C4F5345440094000020B2
:109D4000404D002088000020A4000020A00000203A
:109D50007063622D3E736E645F71756575656C65C9
:109D60006E203E20300000006E6F207365676D65C9
:109D70006E7420746F206672656500007063622DDA
:109D80003E6C697374656E65722D3E6163636570C8
:109D90007420213D204E554C4C000000C168A1426A
:109DA0003FF440AF08460028F8D18AF8009084F8C4
:109DB00014B03868E0603C6001F004FE0FE020461B
:109DC00000F092F82878C00609D5206DA96988426C
:109DD00005D1E06E18B9687840F010006870002076
:109DE000D8E500002DE9F04104000DD0A56F00205A
:109DF0006E7BA067D4F88470002F10D000232A4611
:109E000021462069B84710E017A340F2096222A159
:109E10002BA0F6F7CDFA6FF00F00BDE8F08100231C
:109E20002A462146184600F0E1FC6FF00C0728B1E5
:109E30000D3017D06FF00400A567EEE7B0060FD520
:109E4000208DB0F5066F01D0401C2085D4F88450D9
:109E500035B100231A4621462069A8470D3001D0AC
:109E60000020DAE73846D8E72E2E2F4D6964646C5F
:109E70006577617265732F54686972645F506172AF
:109E800074792F4C7749502F7372632F636F72650B
:109E90002F7463702E6300007463705F70726F6361
:109EA0006573735F726566757365645F6461746121
:109EB0003A20696E76616C6964207063620000000C
:109EC000417373657274696F6E2022257322206658
:109ED00061696C6564206174206C696E652025641D
:109EE00020696E2025730A002DE9F047040006D191
:109EF000E1A340F27B42EDA1F3A0F6F759FA207DF1
:109F0000042806D2DCA340F27C42F9A1EEA0F6F7C9
:109F10004FFAFE4D4FF6FF774FF000062878C00647
:109F20007ED5B4F86020A16D636D686902EB01080D
:109F3000B3EB000C0BD4834202D1AB69CB1A06D42D
:109F4000AB69994210D1E968C98991420CD9E96895
:109F5000C989A4F86010B4F862208A4201D2A4F83A
:109F600062106065A869A065626CA869811A002901
:109F70002EDC698949BBB4F86030A16D19444145B4
:109F800023D1B4F9301000291FDB82421DD194F88F
:109F90004300411CC9B2814201D984F8431094F8AE
:109FA000430003280CD9B4F84810608E084480B2EE
:109FB000884202D3A4F8480003E0A4F8487000E007
:109FC00002D3204600F08CFD8EE084F843608BE0E5
:109FD000012977D4226D821A002A73DC628B530721
:109FE00008D522F004026283B4F84A20A4F848207D
:109FF000A4F86A6084F84260E28FB4F93C3089B218
:10A0000002EBE302A4F8402084F843606064207D02
:10A01000042831D3B4F84800B4F84A20904200E054
:10A0200082E015D2628B120501D5012200E00222E6
:10A03000638E53439AB28A4200D81146014489B2D2
:10A04000814202D3A4F8481016E0A4F8487013E047
:10A05000B4F86A20114489B2914202D3A4F86A107C
:10A0600001E0A4F86A70B4F86A10814204D3091AB6
:10A07000A4F86A10618EE1E7D4E91B31A4A220465E
:10A08000FDF7ACFE20670346A3A22046E16EFDF774
:10A09000A5FEE066216F19B12686267720B105E07E
:10A0A0004FF0FF322286F8E7A4F86860B4F8642025
:10A0B0002B891A44A4F86420628B120514D511B1BF
:10A0C000C86802E00DE038B1C0684068FBF7A6F848
:10A0D000E16C081A002807DC608B20F400606083C4
:10A0E00002E0204600F094FF606BE8B1A16BAA6922
:10A0F000891A19D58A490988081AB4F93C10A0EBC5
:10A10000E10000B2014409B2A187002801DA40420F
:10A1100000B2B4F93E20A0EBA2001044E08700EBAF
:10A12000E100A4F840006663B5F80AC0BCF1000F76
:10A130007ED0207D07287BD2616A6A69DFF8E4A1BE
:10A14000881AA946012849D402EB0C054D1B6D1C49
:10A15000002D43DCDAF80450804635B946A340F2BE
:10A16000945271A158A0F6F723F9B84506D342A33B
:10A1700040F2955270A154A0F6F71AF9DAF80400EB
:10A180001FFA88F7D0460089B84206D23AA340F2B7
:10A1900097526DA14CA0F6F70BF9B8F80810C91B3F
:10A1A000A8F80810D8F804000089C01B81B204E0A8
:10A1B00029816E81381A2D6887B26889B842F7D331
:10A1C00039462846FCF718FE606AC9F81400D8F82A
:10A1D0000C104860616A401A07D593E2501A04D502
:10A1E000608B40F0020060838CE2208D0A460144BF
:10A1F000D9F814004F46411A491C0029EDDC82426F
:10A2000038D1DAF80C0055468089FBF709F8800749
:10A2100000D001202989B846084480B27881218D78
:10A22000814228D2E8688089FAF7FAFFC00700E087
:10A230006DE20ED0E8688089FAF7F2FFC0F34400BF
:10A240004000FAF7EDFFE9688A8922F47C52104356
:10A250008881208D2881E8688089FAF7E1FF8007EE
:10A2600002D52889401E288129896868FCF7E4FC0A
:10A27000E86871E08DE18BE02E2E2F4D6964646CEF
:10A280006577617265732F54686972645F5061729B
:10A2900074792F4C7749502F7372632F636F7265F7
:10A2A0002F7463705F696E2E630000007463705FCB
:10A2B000726563656976653A20696E76616C69647A
:10A2C0002070636200000000417373657274696FEF
:10A2D0006E2022257322206661696C65642061749A
:10A2E000206C696E6520256420696E2025730A0044
:10A2F0007463705F726563656976653A2077726F23
:10A300006E6720737461746500000000A80000206F
:10A31000756E61636B656400756E73656E740000C5
:10A32000940000206C820020696E7365672E702097
:10A33000213D204E554C4C00696E73616E65206F57
:10A3400066667365742100007062756620746F6FB5
:10A350002073686F727421008089FAF761FF8007AB
:10A3600000D001202989084481B2A8F80A10238D61
:10A37000626AD8F814001A440844904208D0AFF238
:10A38000081340F2CB52E9A1AFF2C400F6F710F87F
:10A39000606F002873D0E8688089FAF741FFC00732
:10A3A00004D107E00168616700F01AFE606F0028C1
:10A3B000F8D164E0676F1EE08889FAF731FFC007C3
:10A3C00015D0E8688089FAF72BFF80070FD40120A9
:10A3D000FAF726FFE9688A8910438881FAF720FF97
:10A3E000800700D0012029890844A8F80A003846CF
:10A3F0003F6800F0F5FDDFB3F9683A89D8F814300A
:10A4000048680244B8F80A001844801AD4D5B8F84D
:10A410000A20D8F814108B18FA6852689B1A002B7F
:10A420002CDD501A2881E8688089FAF7F9FE800748
:10A4300002D52889401E288129896868FCF7FCFB21
:10A44000E8688089FAF7ECFE800700D001202989AE
:10A45000084481B2A8F80A10D8F814000844F96832
:10A46000496888420AD0AFF2F01340F2FC5200E093
:10A4700004E0BCA1AFF2B010F5F79AFF6767B8F837
:10A480000A00D8F81410474601446162218D8142C8
:10A4900008D2AFF21C2340F20762C1A1AFF2D8107C
:10A4A000F5F786FF208D7989401A2085204601F036
:10A4B0003BFB6868018909B1F8616E60E8688089D2
:10A4C000FAF7AEFEC00752D0787840F020007870DE
:10A4D0004DE079618089FAF7A3FE800700D0012062
:10A4E0002A89616A114408446062E8688089FAF741
:10A4F00097FE800700D0012029890844218D8842D9
:10A5000008D9AFF28C2340F22B62ADA1AFF2482004
:10A51000F5F74EFFE8688089FAF782FE800700D0E1
:10A52000012029890844218D081A2085204601F040
:10A53000FBFA6968088930B1F86910B1FCF73EF898
:10A5400000E0F9616E60E8688089FAF769FEC0078B
:10A5500008D0787840F020007870207D042801D160
:10A560000720207528686067284600F039FD656F70
:10A5700025B1E868626A41689142AAD0608BC10740
:10A5800002D020F00100CEE040F001006083BDE881
:10A59000F087656F9DB10026C846E9684968814229
:10A5A00012D1BAF80800298988420CD98E4800F0E7
:10A5B000C1FC002807D08EB33060294625E08A48C8
:10A5C00000F0B8FC60679DE016B3F2685268821A2A
:10A5D000012A25D4421A521C002A21DC824800F0AC
:10A5E000A9FC070013D0F068318940684218D8F8F8
:10A5F0001410521A002A05DD081A81B231817068E0
:10A60000FCF71AFB294638463760FEF7DBFA79E09B
:10A61000421A05D5744800F08DFCE8B36067CCE7BA
:10A620002A682E46CABB411A002968DDE86880897D
:10A63000FAF7F6FDC00765D16B4800F07BFC286097
:10A6400050B3E8684646416828890A18D8F81400CB
:10A65000121A002A05DD401A81B229816868FCF7C8
:10A66000EBFA218D606A7269084471891144081AF5
:10A67000002847DD2868C0688089FAF7D1FDC00747
:10A6800013D02868C0688089FAF7CAFDC0F3440077
:10A690004000FAF7C5FD01E030E030E02968C96804
:10A6A0008A8922F47C5210438881A08C218D084431
:10A6B000B18A401A81B22868018128684068FCF795
:10A6C000BBFA2868C0688089FAF7AAFD800700D025
:10A6D000012029680989084480B27081228D616A4D
:10A6E00011447269104488420CD0AFF274434FF4A5
:10A6F000DF620EA1AFF23040F5F75AFE02E015001E
:10A700007FF44BAF2046BDE8F04700F081BC606AA3
:10A7100069690A1A06D4228D1044081A401C0028C0
:10A720007FF735AF608B40F002002FE77463705FF6
:10A73000726563656976653A207365676D656E74E9
:10A74000206E6F74207472696D6D656420636F7222
:10A75000726563746C7920746F207263765F776EB4
:10A76000640A00007463705F726563656976653AB8
:10A77000207365676D656E74206E6F7420747269E6
:10A780006D6D656420636F72726563746C7920749B
:10A790006F206F6F7365712071756575650A0000B4
:10A7A0007463705F726563656976653A207463707F
:10A7B0006C656E203E207263765F776E640A0000DF
:10A7C0007463705F726563656976653A206F6F7355
:10A7D0006571207463706C656E203E207263765FD5
:10A7E000776E640A000000006C82002010B51446E9
:10A7F000080008D0002C10D0218900F04FF8204626
:10A80000FCF748F90AE008A34FF4D36212A119A09B
:10A81000F5F7CEFD6FF00F0010BD0BB1002010BD9D
:10A82000BDE81040FCF786BE2E2E2F4D6964646C87
:10A830006577617265732F54686972645F506172E5
:10A8400074792F4C7749502F7372632F636F726541
:10A850002F7463702E6300007463705F726563769B
:10A860005F6E756C6C3A20696E76616C69642070FD
:10A8700063620000417373657274696F6E202225F4
:10A880007322206661696C6564206174206C696E56
:10A890006520256420696E2025730A0070B50D4679
:10A8A000040003D0207D012809D00FE0BDE87040EE
:10A8B00014A340F2CF321FA124A0F5F779BD11A354
:10A8C00040F2D2322BA121A0F5F772FD218D4FF479
:10A8D0000662481980B2904201D8814201D922858E
:10A8E00000E02085204601F01FF9B0F5067F08D36F
:10A8F000608B40F0020060832046BDE87040FEF7A8
:10A90000E7B970BD2E2E2F4D6964646C6577617256
:10A9100065732F54686972645F50617274792F4C4B
:10A920007749502F7372632F636F72652F74637052
:10A930002E6300007463705F7265637665643A200D
:10A94000696E76616C69642070636200417373653F
:10A950007274696F6E2022257322206661696C65AE
:10A9600064206174206C696E6520256420696E2006
:10A9700025730A00646F6E27742063616C6C207409
:10A9800063705F72656376656420666F72206C69C0
:10A990007374656E2D7063627300000070B50D00F6
:10A9A000044606D1084BFF2208A103F14400F5F745
:10A9B000FFFC002004E0E16FA94200D1E067E468F9
:10A9C000002CF8D170BD0000707D00087463705FCA
:10A9D00072656D6F76655F6C697374656E65723AEA
:10A9E00020696E76616C6964206C697374656E654C
:10A9F000720000002DE9F041040006D11BA340F2D3
:10AA0000C16227A12CA0F5F7D3FC256F6FF00506D6
:10AA10001DB12846FEF784FD10B13046BDE8F08137
:10AA2000286804F16C06206700E03668306850B191
:10AA3000C0684068FAF7F2FB0746E8684068FAF732
:10AA4000EDFB381AF1D430682860356028680021A1
:10AA500008B9A4F8681094F84200FF2802D2401CFC
:10AA600084F8420000206163D8E700002E2E2F4DAD
:10AA70006964646C6577617265732F546869726488
:10AA80005F50617274792F4C7749502F7372632F26
:10AA9000636F72652F7463705F6F75742E6300004F
:10AAA0007463705F7265786D69743A20696E76615F
:10AAB0006C69642070636200417373657274696FBE
:10AAC0006E2022257322206661696C6564206174A2
:10AAD000206C696E6520256420696E2025730A004C
:10AAE00010B5040006D119A340F2F96224A12CA0EC
:10AAF000F5F75EFC206F002827D0A07E400724D405
:10AB00002046FFF777FF00281FD1B4F84810B4F8AB
:10AB10006000814200D208464108A4F84A10608EC5
:10AB2000B1EB400F05D24FF6FF7101EA4001A4F8E6
:10AB30004A1089B200EB40000844A4F84800608B3A
:10AB400040F0040060830020208610BD2E2E2F4D83
:10AB50006964646C6577617265732F5468697264A7
:10AB60005F50617274792F4C7749502F7372632F45
:10AB7000636F72652F7463705F6F75742E6300006E
:10AB80007463705F7265786D69745F666173743A3F
:10AB900020696E76616C6964207063620000000059
:10ABA000417373657274696F6E202225732220666B
:10ABB00061696C6564206174206C696E6520256430
:10ABC00020696E2025730A0010B5040006D109A380
:10ABD00040F2AD6214A11BA0F5F7EAFB204600F09D
:10ABE0009BF8002804D12046BDE8104000F03EB894
:10ABF00010BD00002E2E2F4D6964646C6577617264
:10AC000065732F54686972645F50617274792F4C58
:10AC10007749502F7372632F636F72652F7463705F
:10AC20005F6F75742E6300007463705F7265786D7A
:10AC300069745F72746F3A20696E76616C69642022
:10AC400070636200417373657274696F6E202225B0
:10AC50007322206661696C6564206174206C696E82
:10AC60006520256420696E2025730A0010B5040054
:10AC700006D109A34FF4D36214A11DA0F5F798FBE8
:10AC800094F84200FF2802D2401C84F8420020467B
:10AC9000BDE81040FEF71CB82E2E2F4D6964646C81
:10ACA0006577617265732F54686972645F50617271
:10ACB00074792F4C7749502F7372632F636F7265CD
:10ACC0002F7463705F6F75742E6300007463705F20
:10ACD0007265786D69745F72746F5F636F6D6D69B3
:10ACE000743A20696E76616C69642070636200005A
:10ACF000417373657274696F6E202225732220661A
:10AD000061696C6564206174206C696E65202564DE
:10AD100020696E2025730A002DE9F041040006D158
:10AD20001BA340F2636227A12FA0F5F741FB256F1B
:10AD30006FF005065DB103E0FEF7F2FB38B92D6850
:10AD4000286800282846F7D1FEF7EAFB10B1304604
:10AD5000BDE8F081E06E28600026206FC4E91B0684
:10AD6000608B40F400606083E8684068FAF756FA48
:10AD70000746E8688089FAF753FA800700D0012077
:10AD80002989384408446663E0640020E0E7000055
:10AD90002E2E2F4D6964646C6577617265732F5434
:10ADA000686972645F50617274792F4C7749502FD3
:10ADB0007372632F636F72652F7463705F6F757446
:10ADC0002E6300007463705F7265786D69745F72E2
:10ADD000746F5F707265706172653A20696E76613A
:10ADE0006C69642070636200417373657274696F8B
:10ADF0006E2022257322206661696C65642061746F
:10AE0000206C696E6520256420696E2025730A0018
:10AE100018B1007A08B1FAF7D1BF1046F9F7CCBDE6
:10AE20002DE9FF4F85B01E00DDE91279DDF8508075
:10AE300093468A4606D11AA340F2C47225A12CA0DB
:10AE4000F5F7B6FA002F06D115A340F2C57232A16C
:10AE500027A0F5F7ADFA002546F208045046FAF7A8
:10AE6000DDF91422CDE90224CDE900980346002241
:10AE700029465846FEF702F904000ED001462B463B
:10AE800000220598FEF7F2F9059809B03B463246D4
:10AE90002146BDE8F04FFEF779B909B0BDE8F08F63
:10AEA0002E2E2F4D6964646C6577617265732F5423
:10AEB000686972645F50617274792F4C7749502FC2
:10AEC0007372632F636F72652F7463705F6F757435
:10AED0002E6300007463705F7273743A20696E763B
:10AEE000616C6964206C6F63616C5F697000000065
:10AEF000417373657274696F6E2022257322206618
:10AF000061696C6564206174206C696E65202564DC
:10AF100020696E2025730A007463705F7273743A3F
:10AF200020696E76616C69642072656D6F74655F0F
:10AF30006970000070B5050006D10CA340F2826272
:10AF400016A11DA0F5F734FA0320FAF72FFD04002F
:10AF50000AD004CD95E80B0004C484E80B00241F3C
:10AF6000FBF704FF204670BD002070BD2E2E2F4D34
:10AF70006964646C6577617265732F546869726483
:10AF80005F50617274792F4C7749502F7372632F21
:10AF9000636F72652F7463702E6300007463705F5B
:10AFA0007365675F636F70793A20696E76616C696B
:10AFB0006420736567000000417373657274696F84
:10AFC0006E2022257322206661696C65642061749D
:10AFD000206C696E6520256420696E2025730A0047
:10AFE00010B5040009D0606808B1FBF753FD214695
:10AFF000BDE810400320FAF721BC10BD10B503E0F6
:10B000000468FFF7EDFF20460028F9D110BD0000CD
:10B010002DE9F0414FF0000704003E4606D118A389
:10B0200040F2EA7223A12BA0F5F7C2F90025206DAA
:10B03000FAF7F4F80346002229462046FDF7B8FF48
:10B04000050010D0014633463A462046FEF70EF979
:10B050002246231D29461046FEF798F8618B50B111
:10B0600041F0030109E0608B40F0030060836FF062
:10B070000100BDE8F08121F003016183F9E70000E0
:10B080002E2E2F4D6964646C6577617265732F5441
:10B09000686972645F50617274792F4C7749502FE0
:10B0A0007372632F636F72652F7463705F6F757453
:10B0B0002E6300007463705F73656E645F656D700E
:10B0C00074795F61636B3A20696E76616C696420A4
:10B0D00070636200417373657274696F6E2022251C
:10B0E0007322206661696C6564206174206C696EEE
:10B0F0006520256420696E2025730A0070B505005F
:10B1000006D113A340F2EB321EA125A0F5F750F9AA
:10B11000EC6E0CB909E0044620680028FBD1E06819
:10B120008089FAF77DF8400705D02846BDE87040D1
:10B130000121FCF7BBBC0120FAF772F8E1688A89AB
:10B1400010438881688B40F020006883002070BD28
:10B150002E2E2F4D6964646C6577617265732F5470
:10B16000686972645F50617274792F4C7749502F0F
:10B170007372632F636F72652F7463705F6F757482
:10B180002E6300007463705F73656E645F66696E42
:10B190003A20696E76616C69642070636200000019
:10B1A000417373657274696F6E2022257322206665
:10B1B00061696C6564206174206C696E652025642A
:10B1C00020696E2025730A002DE9FE4FCA4D47F60F
:10B1D000FF7B4FF4FA7AE8684FF00008401CE86003
:10B1E000A878401CA8700027AC6977E1207D002872
:10B1F00006D1C2A340F2BE42CCA1D7A0F5F7D8F841
:10B20000207D012806D1BDA340F2BF42DCA1D2A01F
:10B21000F5F7CEF8207D0A2806D1B8A34FF498623E
:10B22000E2A1CDA0F5F7C4F8A17FA878814202D1B0
:10B230002746E46852E1A0770026207DB146022827
:10B2400005D194F84200062801D301269FE094F826
:10B2500042000C281BD294F89900002841D0206F9E
:10B26000002806D0A5A340F2D442DCA1BAA0F5F78D
:10B270009FF8E06E002806D1A0A340F2D542E4A1D9
:10B28000B5A0F5F795F894F89A000C2801D301269B
:10B2900071E094F89910EC48095C94F898008842A1
:10B2A00002D2401C84F89800C0B2884263D3B4F83C
:10B2B0006010204619B100F06FFA20B107E000F0ED
:10B2C000ADFCE8BB03E02046FDF702FDC0B384F807
:10B2D000988094F8990007284DD2401C84F8990072
:10B2E00049E0B4F93000584501D2401C2086B4F939
:10B2F0003000B4F9401088423DDB2046FFF70CFDDA
:10B3000018B1206FE0B9E06ED0B1207D022813D0D3
:10B3100094F842000C2800D30C20B4F93E10B4F984
:10B320003C2001EBE202C949085C02FA00F05845F2
:10B3300000DB5846A4F840004046A4F8308000E006
:10B3400019E0B4F84820B4F860108A4200D21146DF
:10B350004A08A4F84A20618E4FF6FF7303EA4103BE
:10B360009A4201D2A4F84A30A4F84810A4F86A001E
:10B370002046FFF77BFC207D062808D1A07EC00672
:10B3800005D5206AE968081A282800D9761C607A51
:10B39000000728D5207D042801D0072823D1AC48F8
:10B3A000D4F89410EB680844B0FBFAF2206A181A3B
:10B3B000824203D24FF00109761C14E094F89B20DE
:10B3C00042F29F4312FB03F201EBC201B1FBFAF11F
:10B3D000814208D22046FDF75BF920B994F89B0022
:10B3E000401C84F89B00606F60B1206AE968081A0D
:10B3F000B4F9401001EB4101B0EB410F02D32046FC
:10B40000FCF78AFD207D032802D0092807D00BE035
:10B41000206AE968081A282806D9761C04E0206A00
:10B42000E968081AF028F8D8002E3DD02046D4F854
:10B430009060FEF747F9A8695FB1844206D12FA357
:10B4400040F26D5283A144A0F4F7B2FFE068F860C7
:10B450000AE0A04206D029A340F2715288A13EA082
:10B46000F4F7A6FFE068A861B9F1000F0AD0228BBB
:10B47000E18A201D8DE8070023461846626A216D87
:10B48000FFF7CEFC2046D4F81090E468FCF75EFC91
:10B4900085F8008016B36FF00C014846B047287855
:10B4A00000287FF4A0AE19E02746E468387F401CEE
:10B4B000C0B23877797F884210D387F81C8085F82E
:10B4C0000080D7F88C2032B1394638699047297806
:10B4D0000029E6D110B93846FDF7FAFB002C7FF4BD
:10B4E00085AE0026EC6912E1207D0A2803D003A373
:10B4F00040F2A152DAE0DEE0880000202E2E2F4D2F
:10B500006964646C6577617265732F5468697264ED
:10B510005F50617274792F4C7749502F7372632F8B
:10B52000636F72652F7463702E6300007463705FC5
:10B53000736C6F77746D723A2061637469766520FD
:10B540007063622D3E737461746520213D20434C0D
:10B550004F5345440A000000417373657274696F6C
:10B560006E2022257322206661696C6564206174F7
:10B57000206C696E6520256420696E2025730A00A1
:10B580007463705F736C6F77746D723A206163746B
:10B59000697665207063622D3E7374617465202145
:10B5A0003D204C495354454E0A0000007463705FBF
:10B5B000736C6F77746D723A20616374697665207D
:10B5C0007063622D3E737461746520213D2054497F
:10B5D0004D452D574149540A000000007463705FC7
:10B5E000736C6F7774696D723A20706572736973EA
:10B5F00074207469636B696E672077697468206969
:10B600006E2D666C69676874206461746100000067
:10B610007463705F736C6F7774696D723A207065D4
:10B620007273697374207469636B696E67207769DC
:10B63000746820656D7074792073656E642062751E
:10B6400066666572000000009FC10008D4C1000852
:10B65000B84C0A007463705F736C6F77746D723AE4
:10B66000206D6964646C652074637020213D2074D2
:10B6700063705F6163746976655F70636273000015
:10B680007463705F736C6F77746D723A2066697261
:10B69000737420706362203D3D207463705F61634A
:10B6A000746976655F706362730000001AA1AFF27F
:10B6B0005810F4F77DFE216AE868401AF02812D984
:10B6C0002046FDF7FFFFE86986B1844208D1AFF25A
:10B6D000D41340F2AF521CA1AFF28410F4F768FE0D
:10B6E000E068F0600FE02646E46810E0A04208D071
:10B6F000AFF2F81340F2B3521DA1AFF2A410F4F769
:10B7000057FEE068E8612046E468FCF71FFB002C68
:10B710007FF4EAAEBDE8FE8F7463705F736C6F7781
:10B72000746D723A2054494D452D5741495420704B
:10B7300063622D3E7374617465203D3D2054494D14
:10B74000452D5741495400007463705F736C6F77E7
:10B75000746D723A206D6964646C65207463702046
:10B76000213D207463705F74775F706362730000C3
:10B770007463705F736C6F77746D723A2066697270
:10B78000737420706362203D3D207463705F747732
:10B790005F706362730000002DE9F84F0F460500EB
:10B7A00006D157A340F24B3262A16BA0F4F700FE22
:10B7B000EC6E002C7ED0002F10D02089B8427AD9B0
:10B7C000688EB84206D24EA340F25B326CA162A0F2
:10B7D000F4F7EEFD208900280BD011E048A340F2D9
:10B7E00053326BA15CA0F4F7E3FD6FF00500BDE8F8
:10B7F000F88F43A34FF457726EA157A0F4F7D8FD0A
:10B8000094F80AB05FEACB7001D0042600E000266D
:10B8100020894FF42072C01B1FFA80F808EB060045
:10B8200081B23620FAF73CFD5FEA000A65D0606815
:10B8300022890189891A39448BB2DAF80410424608
:10B840003144FBF79BF8404554D1E0688089F9F713
:10B85000E7FC00F03F064FF00009300703D526F063
:10B8600008064FF00809F00703D026F0010649F05A
:10B870000109E0684068F9F7D1FCC3194A4651460E
:10B880002846CDF800B0FBF7F5FF070032D060681E
:10B89000FAF72CFF35F8661F081A288060680289BD
:10B8A000A2EB080189B2FBF7C7F92189A1EB0800D7
:10B8B000208101E021E01BE03046F9F7B1FCE168AE
:10B8C0008A89104388816068FAF710FF2988084444
:10B8D00028807868FAF70AFF2988084425F866095D
:10B8E000206838602760386810B90020A5F8680023
:10B8F00000207CE75046FBF7CDF84FF0FF3076E7AD
:10B900002E2E2F4D6964646C6577617265732F54B8
:10B91000686972645F50617274792F4C7749502F57
:10B920007372632F636F72652F7463705F6F7574CA
:10B930002E6300007463705F73706C69745F756E62
:10B9400073656E745F7365673A20696E76616C69C2
:10B950006420706362000000417373657274696FE4
:10B960006E2022257322206661696C6564206174F3
:10B97000206C696E6520256420696E2025730A009D
:10B9800073706C6974203C3D206D7373000000007F
:10B9900043616E27742073706C6974207365676DE2
:10B9A000656E7420696E746F206C656E67746820B4
:10B9B00030000000757365672D3E6C656E203E207B
:10B9C000300000000848816800290CD10749084A66
:10B9D00009681268114306D00121816000220549DF
:10B9E000FA20FBF749BB7047CC000020A0000020E4
:10B9F000A40000205DBD00083EB51D4C0546207822
:10BA0000400722D4002D06D11AA340F2EE2226A12F
:10BA10002DA0F4F7CDFC2078810717D5696A6069FD
:10BA2000421A18D42A8D1144411A002913DCE16806
:10BA30002F4B0A8849880093CDE9011261891B1DAB
:10BA400042182846A169FFF7EBF93EBDC00702D0B6
:10BA500028480068286260890028F6D0688B40F08A
:10BA6000020068832846BDE83E40FDF731B900007A
:10BA7000A80000202E2E2F4D6964646C65776172DA
:10BA800065732F54686972645F50617274792F4CCA
:10BA90007749502F7372632F636F72652F746370D1
:10BAA0005F696E2E630000007463705F74696D657A
:10BAB000776169745F696E7075743A20696E76613A
:10BAC0006C69642070636200417373657274696F9E
:10BAD0006E2022257322206661696C656420617482
:10BAE000206C696E6520256420696E2025730A002C
:10BAF000504D00209400002010B5FCF7F1F80548E7
:10BB00004178491C4170C80703D0BDE81040FFF7D9
:10BB10005BBB10BD880000200248417841F0100155
:10BB200041707047A800002070B5040006D115A32D
:10BB300040F2A6321FA128A0F4F73AFC258D626AD4
:10BB4000638E51194FF48666E06AB34200D93346DA
:10BB50000344CB1A02D46585081A70BD111A002956
:10BB600002DD002060850BE0851AB5F5803F06D325
:10BB700004A340F2B63222A117A0F4F719FC6585A0
:10BB8000002070BD2E2E2F4D6964646C6577617244
:10BB900065732F54686972645F50617274792F4CB9
:10BBA0007749502F7372632F636F72652F746370C0
:10BBB0002E6300007463705F7570646174655F72FA
:10BBC00063765F616E6E5F776E643A20696E766150
:10BBD0006C69642070636200417373657274696F8D
:10BBE0006E2022257322206661696C656420617471
:10BBF000206C696E6520256420696E2025730A001B
:10BC00006E65775F7263765F616E6E5F776E6420DC
:10BC10003C3D203078666666660000002DE9F047FE
:10BC200004004FF0000906D12CA340F64F0238A1C2
:10BC300040A0F4F7BDFBE56E35B394F89A00FF28F9
:10BC400002D2401C84F89A00E8688089F9F7E8FA83
:10BC5000C00701D02889D0B100260122E8684946F2
:10BC600043682046FDF7A4F95FEA000812D0D8F82F
:10BC700004100F468EB11120F9F7D2FAB98921F4D8
:10BC80007C510843B88111E00020BDE8F08701260F
:10BC90000022E3E74FF0FF30F7E768682B891431A3
:10BCA0000289D21A93B20122FAF768FEE868406866
:10BCB000F9F7B4FA216D401C091A00D520654B46EE
:10BCC000002241462046FDF7D1FA2246231D414677
:10BCD000BDE8F0471046FDF759BA00002E2E2F4D53
:10BCE0006964646C6577617265732F546869726406
:10BCF0005F50617274792F4C7749502F7372632FA4
:10BD0000636F72652F7463705F6F75742E630000CC
:10BD10007463705F7A65726F5F77696E646F775F67
:10BD200070726F62653A20696E76616C696420702A
:10BD300063620000417373657274696F6E2022251F
:10BD40007322206661696C6564206174206C696E81
:10BD50006520256420696E2025730A0010B5FFF761
:10BD6000CBFE0848084900680968084306D000224D
:10BD7000BDE810400549FA20FBF77EB904490020D0
:10BD8000886010BDA0000020A40000205DBD000858
:10BD9000CC00002010B5F4F759FA0349C0F30D00A8
:10BDA00000F54040088010BDD80000202DE9F04F7C
:10BDB00087B08946070005D14AA3CF2255A15BA0D1
:10BDC000F4F7F6FAB9F1000F05D146A3D02261A12C
:10BDD00056A0F4F7EDFA788908287CD3644D7C6886
:10BDE00029686869F8F7C0F902902088F9F718FA0D
:10BDF00000906088F9F714FADFF878B100268246DF
:10BE0000B046DBF8044032E0618A51452DD1494605
:10BE10002046029A00F0BEF838B3207C400711D4C7
:10BE2000B8F1000F0DD0029860B16869401C09D1CB
:10BE3000D8F80010D9F80400814203D0216881426B
:10BE400000D1A046A18A009881420ED1606810B14D
:10BE50002969884209D136B1E068F060DBF8041046
:10BE6000E160CBF8044024B10BE02646E468002CE6
:10BE7000CAD15FEA080404D1D9F80400696988428C
:10BE800029D108213846FAF7B7FF38B115A34FF486
:10BE9000B87239A125A0F4F78BFA1CE054B1A5695A
:10BEA000CDB1334B3A4610332146E069A84707B07D
:10BEB000BDE8F08F029870B9287DC0F303100E28FA
:10BEC00009D0A889083001B23846FAF79DFE03214F
:10BED0003846F7F7C4FF07B03846BDE8F04FFAF729
:10BEE000D9BD00002E2E2F4D6964646C6577617298
:10BEF00065732F54686972645F50617274792F4C56
:10BF00007749502F7372632F636F72652F7564705A
:10BF10002E6300007564705F696E7075743A2069F5
:10BF20006E76616C6964207062756600417373653A
:10BF30007274696F6E2022257322206661696C65B8
:10BF400064206174206C696E6520256420696E2010
:10BF500025730A007564705F696E7075743A2069A4
:10BF60006E76616C6964206E65746966000000001D
:10BF7000404D0020D8000020706275665F72656DCC
:10BF80006F76655F686561646572206661696C657E
:10BF9000640A000070B516460D46040005D116A3CC
:10BFA000872221A129A0F4F703FA002D05D112A3BD
:10BFB000882230A125A0F4F7FBF9217A374831B166
:10BFC000426892F83020521CD2B2914212D14EB146
:10BFD00074B1216861B14069421C09D0AA6811405E
:10BFE000104003E024B1216811B14069814201D1C0
:10BFF000012070BD002070BD2E2E2F4D6964646C31
:10C000006577617265732F54686972645F506172FD
:10C0100074792F4C7749502F7372632F636F726559
:10C020002F7564702E6300007564705F696E7075A3
:10C03000745F6C6F63616C5F6D617463683A2069F3
:10C040006E76616C69642070636200004173736591
:10C050007274696F6E2022257322206661696C6597
:10C0600064206174206C696E6520256420696E20EF
:10C0700025730A007564705F696E7075745F6C6F0C
:10C0800063616C5F6D617463683A20696E76616CA0
:10C090006964206E6574696600000000404D0020F0
:10C0A00010B5002813D00268002A10D000290ED045
:10C0B0000A68002A0BD0064A526806E01368046832
:10C0C000A34201D10B681360D268002AF6D110BDDB
:10C0D000D80000204FF04070E1EE100A70470000D9
:10C0E00020060C0040010020180000200000000085
:10C0F0000000000001020304060708090000000018
:10C1000001020304FFFFFFFFFFFF0000000000002B
:10C1100020000400AB530020540000209C000500C8
:10C120002E540020580000201C0008003D5700201D
:10C130005C0000201000100020580020600000204B
:10C1400020000500235900206400002018000F0083
:10C15000C65900206800002010000300315B002059
:10C160006C00002010001000645B002070000020B4
:10C1700060021000675C00207400002010C10008FD
:10C180001CC1000828C1000834C1000840C10008D3
:10C190004CC1000858C1000864C1000870C1000803
:10C1A00003060C183060780040C2000868C200081E
:10C1B00088C2000848C2000834C200081CC2000837
:10C1C00028C200087CC2000854C200085CC20008F3
:10C1D00070C20008010203040506070707070707E6
:10C1E000070000009C00002098000020A000002014
:10C1F000A4000020FA000000F9BA0008E8030000DB
:10C20000C54F0008E8030000053A000800000000E0
:10C210003A7474003A7474003A74740046494E5F7C
:10C22000574149545F31000046494E5F57414954D8
:10C230005F32000045535441424C49534845440045
:10C24000434C4F534544000053594E5F52435644AC
:10C2500000000000434C4F53494E47004C4153549B
:10C260005F41434B000000004C495354454E0000D1
:10C2700054494D455F57414954000000434C4F53CA
:10C28000455F57414954000053594E5F53454E5442
:10C29000000000007463705F656E71756575655FA1
:10C2A000666C6167733A206E6565642065697468C1
:10C2B0006572205443505F53594E206F722054438F
:10C2C000505F46494E20696E20666C616773202876
:10C2D00070726F6772616D6D65722076696F6C61E7
:10C2E0007465732041504929000000006E6574692F
:10C2F000662D3E6877616464725F6C656E206D7553
:10C300007374206265207468652073616D652061B7
:10C3100073204554485F4857414444525F4C454E52
:10C3200020666F72206574686172702100000000E1
:10C3300050C3000800000020F8000000C4010008FD
:10C3400048C40008F8000020B88A0000E001000896
:10C3500000000000351500082B15000861150008C5
:10C36000451500082F15000800000000000000001F
:10C3700000000000000000000000000000000000BD
:10C38000000000000000000001000000100000009C
:10C39000000000000024F400000000000000000085
:10C3A000000000000000000000000000000000008D
:10C3B000000000000000000000000000000000007D
:10C3C000000000000000000000000000000000006D
:10C3D00000000000000000000000000000C000009D
:10C3E0006E190000000000000000000000000000C6
:10C3F000000000000000000000000000000000003D
:10C40000000000000000000000000000000000002C
:10C41000000000000000000000000000000000001C
:10C42000000000000000000000C00000000000004C
:10C4300000000000000000000000000000000000FC
:08C440000000000000000000F4
:040000050800018965
:00000001FF
